:1000000000400020AD420000ED420000EF42000041
:1000100000000000000000000000000000000000E0
:10002000000000000000000000000000F14200009D
:100030000000000000000000F3420000F542000054
:10004000F7420000F7420000E14A0000F7420000DA
:10005000F742000000000000F7420000F7420000F5
:10006000F742000025450000F7420000F74200007B
:10007000F7420000F7420000F7420000F74200009C
:10008000F7420000854B0000F7420000F7420000F5
:10009000F7420000F7420000F7420000F74200007C
:1000A000F7420000F74200000000000000000000DE
:1000B0000000000000000000000000000000000040
:1000C000054B0648033310B51B1A062B03D9044B06
:1000D000002B00D0984710BD3001002030010020D7
:1000E000000000000648074910B5091A8910CB0F17
:1000F0005918491003D0044B002B00D0984710BD6D
:1001000030010020300100200000000010B5074C35
:100110002378002B09D1FFF7D3FF054B002B02D02A
:10012000044800E000BF0123237010BD300100200F
:100130000000000020710000094B10B5002B03D017
:100140000849094800E000BF08480368002B02D1B5
:10015000FFF7C8FF10BD064B002BF9D09847F7E713
:100160000000000034010020207100002C0100205C
:1001700000000000164B002B00D1144B9D4640227E
:1001800092029A1A924600218B460F461348144A4F
:10019000121A04F066FF0F4B002B00D098470E4B4D
:1001A000002B00D098470020002104000D000D48CE
:1001B000002802D00C4800E000BF04F00FFF200030
:1001C000290004F0A5FC04F0E3FEC046000008008E
:1001D000004000200000000000000000300100206E
:1001E000901F0020000000000000000001230340D9
:1001F0000200181E04D1042A03D91068000900E087
:100200000020704710B50400FFF7F0FF0300012045
:10021000002B0BD0013B9B00181DE2181279002A1D
:1002200003D001338342F8D100E0180010BD012251
:10023000016810B5114201D0002903DA102001F045
:10024000F9FD03E04910062001F0BEFE10BD016873
:1002500010B5CB0701D5002903DA102001F0EAFD23
:1002600006E04910033189100022052001F0ACFEA0
:1002700010BD70B50568AB0728D1042D26D90F2312
:100280002A6846681340062B09D12800FFF7AEFF05
:10029000012383421DDC9A00AE500133F9E7052BA0
:1002A00014D1F30703D4132001F0C4FD12E076103B
:1002B000FF2EF8D82800FFF799FF2C1D230080009F
:1002C0002018984205D91E700133FAE70B2001F07F
:1002D000B1FD002070BD70B50468E30701D41120A2
:1002E0002DE04568AB0729D1042D27D90F262B68AF
:1002F00064101E40062E0BD1002C04DD2800FFF7F1
:1003000075FF844201DD122019E0A400605918E055
:10031000331F012B12D82800FFF768FF8000042E3E
:1003200002D12800FFF76EFF002CECDDA042EADBD3
:1003300001232C19E0784000184302E00B2001F063
:1003400079FD70BDF8B5012304681C4201D111206C
:100350002FE00325466835402AD1042E28D90F23E3
:100360003268641087681340062B0BD1002C04DD23
:100370003000FFF73BFF844201DD122019E0A400AA
:10038000A75113E0052B13D1002CF6DD3000FFF749
:100390002DFF80008442F0DC01231F4201D1132095
:1003A00007E07F10FF2FFAD83419E770280002E029
:1003B0000B2001F03FFDF8BD006810B5830717D191
:1003C000042815D90F2302681340062B02D1FFF72A
:1003D0000DFF0BE0052B05D1FFF708FFC00001233F
:1003E000184308E0042B03D1FFF70CFF4000F6E7A9
:1003F0000B2001F01FFD10BD10B503240068044060
:1004000006D1042804D90F2302681340042B01D01D
:100410000E2011E001F014FE0378233B59425941AC
:1004200010224018210005F0E3FA80239B05C21832
:10043000054B9A4203D9142001F0FCFC02E0012391
:100440004000184310BDC046FFFFFF3F10B5012418
:100450000368234202D04268224203D10D2001F0FA
:10046000E9FC08E004495B1052101B070A401343E3
:1004700018684000204310BDFCFFFF0F01210368F6
:1004800010B50B4205D042680A4202D0806808428B
:1004900003D10D2001F0CEFC08E005495B1052109D
:1004A0001B070A40401013431860002010BDC046CF
:1004B000FCFFFF0F012303400200181E01D0501063
:1004C00002E00D22014B1A707047C0464C0100201B
:1004D000012303400200181E04D1042A03D9106826
:1004E000000900E00020704770B50D000400FFF720
:1004F000EFFF86002800FFF7EBFF830000209E42FD
:100500000ED1231D9E1904351A009E4207D9297861
:100510001278013301358A42F6D0002000E0012034
:1005200070BD0000F0B585B00393019002912D4E8F
:100530002D4B002A02D002223270013A00251A60A7
:100540001B68F554019B9D424ADA029AAB00D058D1
:10055000254B1C68C8239B0037191C1B012318421C
:1005600002D04310214A1FE0214A002802D004286B
:1005700005D1204A2100380005F03AF918E0042896
:1005800010D90F2302681340042B04D101F058FD49
:10059000194A030008E0062B05D1FFF799FF174A17
:1005A000030001E00123164A2100380005F020F97C
:1005B000300005F083F9039B0B4A002B01D110603A
:1005C0000CE0019B013B9D42F9DA0E4B9842F6DCB0
:1005D000431C1360202232540022F2540135B1E74B
:1005E00005B0F0BD5801002054010020BD65000099
:1005F0009065000096650000046A00009B6500009D
:10060000AC6500001F030000C368F0B59D0083685F
:1006100087B05D19030018330393036902909C00AF
:10062000039B1F1943699E000093039B9E19D44BA3
:100630001B78002B0FD17F222B68D2491C1213404C
:100640009B005B5800960435019234E0CC4B1B783C
:10065000002B28D0009E029BC94C9B6821780093F8
:10066000EA1A029B92109B7812021A43029B587856
:1006700002F0FCFA0023029A237013700096029B8A
:10068000039A9B68ED1A0193029BAD10DD60039BFA
:10069000FC1A029BA4101C61009B9B1A029A9B10DF
:1006A000536101F0C1FB2B68019A1C121340B54A3B
:1006B0009B009B5804359F46029B587802F0CEFA67
:1006C000A6E2039B3A1DD11AAD4B8B2903DD1A22FA
:1006D000009E1A70BFE71B783C60002B02D0009E82
:1006E0001700B8E72B6801991C120B40A5499B0025
:1006F0005B5817000435DEE7039B3A1DD11AA04B67
:100700008B2903DD1A22009E1A70A4E728681B7843
:10071000291D3860002B03D0009E17000D009AE7BA
:100720006B6801991C120B4096499B005B5817009F
:100730000835C0E7039B3A1DD11A914B8B2903DD85
:100740001A22009E1A7086E7A4001B782C193C60C0
:10075000002B02D0009E17007DE72B6801991C1228
:100760000B4088499B005B5817000435A3E7039BA7
:100770003A1DD11A824B8B2903DD1A22009E1A7072
:1007800069E78148A40021581B783960002B02D00A
:10079000009E17005FE72B6801991C120B407949F6
:1007A0009B005B581700043585E73A1F764B1168AC
:1007B000A400E150724B1B78002B02D0009E170062
:1007C00049E72B6801991C120B406E499B005B584E
:1007D000170004356FE76C4BA600F058FFF76AFE70
:1007E000043F04003868FFF765FE24180120664BBB
:1007F00064000443F450624B1B78002B01D0009E30
:1008000029E72B68019A1C1213405E4A9B009B58F3
:10081000043550E7039B3A1DD11A594B8B2903DD50
:100820001A22009E1A7016E70098039C0121A0422C
:1008300002D901000C3909681B783960002B02D0FD
:10084000009E170007E72B6801991C120B404D49C9
:100850009B005B58170004352DE7039B3A1DD11A06
:10086000474B8B2903DD1A22009E1A70F3E600998C
:10087000039881420AD90B000C3B1B6843495B106B
:100880006418E41A009BA400E35802E018211970D0
:1008900000233B603A4B1B78002B02D0009E1700D0
:1008A000D9E62B6801991C120B4036499B005B5816
:1008B00017000435FFE6009B039A93420CD90C3BCA
:1008C0001968324B3A1FE3184910591A1068009BF7
:1008D0008900C850170002E01822294B1A70284BD3
:1008E0001B78002B01D0009EB5E62B68019A1C12E4
:1008F0001340244A9B009B580435DCE6009B039A76
:10090000934220D9009E214B0C3EE3180493336898
:10091000049A5B10D31A009A9B009858FFF7CAFDFF
:100920003C1F05902068FFF7C5FD3168049B491006
:10093000591A059B009A1B1801205B00890003438C
:100940008B50270002E018220D4B1A700C4B1B78BD
:10095000002B01D0009E7EE62B68019A1C121340EA
:10096000084A9B009B580435A5E6039B3A1DD11A03
:10097000034B8B290CDD1A22009E1A706BE6C046D1
:100980004C010020D0650000701E0020FDFFFF3FDD
:100990000099A40061581B783960002B02D0009E9A
:1009A000170058E62B6801991C120B40D0499B0098
:1009B0005B58170004357EE63A1F009B1168A400BF
:1009C000E150CC4B1B78002B02D0009E170042E672
:1009D0002B6801991C120B40C5499B005B581700FE
:1009E000043568E6009BA4001C192368043F38689E
:1009F0005E10FFF75FFD36180120BE4B76001B78B6
:100A000006432660002B01D0009E24E62B68019A45
:100A10001C121340B64A9B009B5804354BE6039BBF
:100A2000A4003F1BB34CBB420DD82378002B01D050
:100A3000009E10E62B68019A1C121340AC4A9B00E2
:100A40009B58043537E6AC4801F070FA2378002B48
:100A500001D0009EFFE52B68019A1C121340A44AA6
:100A60009B009B58043526E6A300ED18002C00DA05
:100A700005E6A04B1B78002B01D0009EEBE52B6810
:100A8000019A1C1213409A4A9B009B58043512E6A7
:100A90003A1F1368042B03D1A300ED18002C18DBB8
:100AA000944B1B78002B02D0009E1700D3E52B68D7
:100AB00001991C120B408E499B005B5817000435AE
:100AC000F9E53A1F1368002B05D1A300ED18002C9F
:100AD00001DA1700D3E5874B1B78002B02D0009E6C
:100AE0001700B8E52B6801991C120B4080499B0048
:100AF0005B5817000435DEE53A1F13685B10013BB5
:100B0000002B06DD01215B00A4000B432D191360AF
:100B1000B5E5784B17001B78002B01D0009E9AE5B5
:100B20002B68019A1C121340714A9B009B58043594
:100B3000C1E53A00039B0C32D31A8B2B04DD1A2239
:100B40006C4B009E1A7086E5FF2361005B000B4032
:100B500001210B433B60029B03989B682412049382
:100B6000ED1A029BAD109B782D021D43009B8D401A
:100B70001B1A9B108B400B43BB60029B0D437D6097
:100B80009C70E4B25D4BE4000299E35816008B6060
:100B900058490978002903D008331D0017005AE589
:100BA0001D0001999B680C351C120B4050499B009D
:100BB0005B58009217007EE53B1F1E68039A009B5E
:100BC000934229D10A20F30716D4B3070DD1042E7E
:100BD0000BD90F2332681340042B06D1300001F0EB
:100BE0002FFA04F06BFE063006E00720042E03D037
:100BF000002E01D080208000643001F035FE0028F6
:100C000001D101F095F8029B3100587802F040F8CC
:100C10000023029A137032E5009B009A0C3B1B687C
:100C200002995B109B005B421C00D3180C3B1E60BA
:100C30001300083B1B68083C17195A108A70D2B27F
:100C40002E49D2005B0055589B0A029A9B00956082
:100C5000ED18009B043B1E68039B7610B6009E199E
:100C6000244B1B78002B00D0F5E42B68019A1C1252
:100C700013401F4A9B009B58009604351BE53B1F01
:100C80001868FFF717FCA40006003F1B1E2829DC8C
:100C900000280EDC174B1B78002B01D0009EDAE4F5
:100CA0002B68019A1C121340114A9B009B58043573
:100CB00001E502F035FA083E361802F031FA104B21
:100CC000801B9842F9D80B4B1B78002B01D0009E5B
:100CD000C1E42B68019A1C121340054A9B009B58E3
:100CE0000435E8E40123029A137002F019FA2CE0AB
:100CF000D06500004C010020C0650000781600207F
:100D00009F8601003B1F1868FFF7D4FBC84BA40067
:100D100006003F1B98421DDC00280EDCC54B1B78EB
:100D2000002B01D0009E96E42B68019A1C12134000
:100D3000C14A9B009B580435BDE40123029A1370FD
:100D400002F0EEF9FA239B005E431138029B36183D
:100D50005E6094E40223029A137002F0EBF9F5E767
:100D6000A300FF1A002320001A003900FFF7DAFB66
:100D7000B24EB34C3168200001F010FF3168200002
:100D800001F08DFFAB4B1B78002B01D0009E62E47D
:100D90002B68019A1C121340A74A9B009B580435EC
:100DA00089E4A44BA4001B783F1B002B01D0009EBC
:100DB00051E42B68019A1C1213409F4A9B009B58D8
:100DC000043578E401F096FD01F02EF83B1F186819
:100DD000002823D1083B1868C30701D5401016E04E
:100DE00083070FD104280DD90F2302681340062B67
:100DF00002D1FFF76DFB0AE0052B03D1FFF768FB7B
:100E0000800004E019228B4B009E1A7023E43A0004
:100E100001214300083A0B43136001E04010013800
:100E2000002832DD012243001343391F0B603B00D1
:100E3000083B1B681341181A3B000C3B1B6813420C
:100E400003D08018A400904015E0990717D1042B17
:100E500015D90F211E683140062906D101308000C6
:100E6000C358009AA400A35010E0052907D1181810
:100E70000079A4004000009B1043E05006E01922D6
:100E80006C4B009E1A70FFF7E6FB0435694B1B782C
:100E9000002B02D0009EFFF7DEFB2B68019A1C128C
:100EA0001340654A9B009B580435FFF704FCA300E0
:100EB000039AFB189B1A8B2B01DC002205E01A22F7
:100EC0005C4B009E1A70FFF7C6FB631E002C03DD0F
:100ED0003A601C000437F8E7564B1B78002B02D011
:100EE000009EFFF7B8FB2B68019A1C121340524A70
:100EF0009B009B580435FFF7DEFB3B00083B18685E
:100F0000FFF7D8FA3B1F04901868FFF7D3FA049A4A
:100F1000A600BC1B0023824200DA04332360454B49
:100F2000BC1B1B78271D002B02D0009EFFF793FBF4
:100F30002B68019A1C1213403F4A9B009B580435B2
:100F4000FFF7B9FBA300FE1A04933B00083B1868A7
:100F5000FFF7B0FA3B1F04001868FFF7ABFAE20F87
:100F6000C317A04253419B003360049BFC1A314BD2
:100F7000271D1B78002B02D0009EFFF76CFB2B680F
:100F8000019A1C1213402C4A9B009B580435FFF712
:100F900092FB3B00083B18683B1F1968A30088427E
:100FA00002D1FB1A042222E004281ED90122104299
:100FB00001D0114219D10326304215D10F23026806
:100FC0001A40042A10D131420ED104290CD90A68E2
:100FD0001340042B08D1FFF787FA431E9841A6005F
:100FE000BE1B8000306003E0A3000022FB1A1A60E1
:100FF000104BA4001B783C1B271D002B02D0009E29
:10100000FFF729FB2B68019A1C1213400A4A9B0028
:101010009B580435FFF74FFB3B00083B18683B1F0C
:101020001968A30088420DD1FB1A00222EE0C046A9
:10103000E70300004C010020D065000054010020AF
:101040005801002004281FD90122104201D011426A
:101050001AD10326304216D10F2302681A40042AFF
:1010600011D131420FD104290DD90A681340042B44
:1010700009D1FFF739FA030058425841A600BE1BB8
:101080008000306003E0A3000422FB1A1A60EA4BE0
:10109000A4001B783C1B271D002B02D0009EFFF7ED
:1010A000DAFA2B68019A1C121340E44A9B009B5801
:1010B0000435FFF700FBA300FE1A04933B00083B36
:1010C0001868FFF7F7F93B1F04001868FFF7F2F9FB
:1010D000E217C30F844253419B003360049BFC1A08
:1010E000D54B271D1B78002B02D0009EFFF7B3FACB
:1010F0002B68019A1C121340D04A9B009B58043560
:10110000FFF7D9FA3B00083B1868FFF7D3F93B1FFC
:1011100004901868FFF7CEF9049AA600BC1B0023C0
:10112000824200DD04332360C34BBC1B1B78271DA8
:10113000002B02D0009EFFF78EFA2B68019A1C123A
:101140001340BE4A9B009B580435FFF7B4FA3B1F7F
:101150001B68B94AA400042B02D13B1B002103E009
:10116000002B03D104213B1B196001E00C231370F9
:1011700013783C1B271D002B02D0009EFFF76BFA53
:101180002B68019A1C121340AC4A9B009B580435F3
:10119000FFF791FAA300FC1A04933B00083B186880
:1011A000FFF788F93B1F06001868FFF783F9361828
:1011B0000120049B760006432660FC1A9E4B271DE7
:1011C0001B78002B02D0009EFFF745FA2B68019A8E
:1011D0001C121340994A9B009B580435FFF76BFA89
:1011E000A300FE1A04933B00083B1868FFF762F95E
:1011F0003B1F04001868FFF75DF9241A0120049BC7
:10120000640004433460FC1A8B4B271D1B78002BB1
:1012100002D0009EFFF71FFA2B68019A1C121340A0
:10122000864A9B009B580435FFF745FAA300FC1A39
:1012300004933B00083B1868FFF73CF93B1F06008E
:101240001868FFF737F946430120049B76000643F0
:101250002660FC1A784B271D1B78002B02D0009EBD
:10126000FFF7F9F92B68019A1C121340734A9B008F
:101270009B580435FFF71FFA3B00083B1868FFF73F
:1012800019F93B1F04901868FFF714F9010004983E
:1012900003F046FD012340001843674BA4001B7870
:1012A0003E1B3060371D002B02D0009EFFF7D3F9A4
:1012B0002B68019A1C121340604A9B009B5804350E
:1012C000FFF7F9F93B00083B1868FFF7F3F83B1FFD
:1012D00004901868FFF7EEF80100049803F006FE8A
:1012E000012349001943544BA4001B783E1B316075
:1012F000371D002B02D0009EFFF7ADF92B68019A35
:101300001C1213404D4A9B009B580435FFF7D3F93C
:101310003B1F1868FFF7CEF8C317C01858400123C9
:1013200040001843444BA4001B783E1B3060371D1F
:10133000002B02D0009EFFF78EF92B68019A1C1239
:1013400013403E4A9B009B580435FFF7B4F9A300B5
:10135000FE1A05933068012C03D1FFF7ABF8049017
:1013600008E0FFF7A7F804007068FFF7A3F8013062
:10137000031B0493049B002B01DC0123049304F062
:10138000E9F9049903F0B2FD0C190121059B6400F1
:101390000C433460FC1A284B271D1B78002B02D00D
:1013A000009EFFF758F92B68019A1C121340234A3C
:1013B0009B009B580435FFF77EF9A4003E1B3000CC
:1013C000FFF71AF81C4B30601B78371D002B02D03A
:1013D000009EFFF740F92B68019A1C121340174A30
:1013E0009B009B580435FFF766F9A300FE1A04938F
:1013F0003B00083B1868FFF75DF83B1F04001868C6
:10140000FFF758F804400120049B64000443346053
:10141000FC1A094B271D1B78002B02D0009EFFF7FA
:101420001AF92B68019A1C121340044A9B009B581E
:101430000435FFF740F9C0464C010020D06500009C
:10144000A300FC1A04933B00083B1868FFF732F82E
:101450003B1F06001868FFF72DF806430120049B88
:10146000760006432660FC1ADD4B271D1B78002BF7
:1014700002D0009EFFF7EFF82B68019A1C12134070
:10148000D84A9B009B580435FFF715F9A300FC1AB6
:1014900004933B00083B1868FFF70CF83B1F06005D
:1014A0001868FFF707F846400120049B76000643C2
:1014B0002660FC1ACA4B271D1B78002B02D0009E09
:1014C000FFF7C9F82B68019A1C121340C54A9B000C
:1014D0009B580435FFF7EFF83B1F1868FEF7EAFF4B
:1014E000C043012340001843BD4BA4001B783E1BA2
:1014F0003060371D002B02D0009EFFF7ACF82B6840
:10150000019A1C121340B74A9B009B580435FFF701
:10151000D2F8A300FE1A04933B00083B1868FEF7BC
:10152000C9FF3B1F04001868FEF7C4FF8440012375
:1015300064001C43049B3460FC1AA94B271D1B78D4
:10154000002B02D0009EFFF786F82B68019A1C1230
:101550001340A44A9B009B580435FFF7ACF8A30046
:10156000FE1A04933B00083B1868FEF7A3FF3B1FDD
:1015700004001868FEF79EFF0441012364001C4329
:10158000049B3460FC1A964B271D1B78002B02D05D
:10159000009EFFF760F82B68019A1C121340914AD5
:1015A0009B009B580435FFF786F8A4003E1B3000D3
:1015B000FEF73DFE8A4B30601B78371D002B02D0B2
:1015C000009EFFF748F82B68019A1C121340854AC9
:1015D0009B009B580435FFF76EF8A4003E1B3000BB
:1015E000FEF735FE7E4B30601B78371D002B02D096
:1015F000009EFFF730F82B68019A1C121340794ABD
:101600009B009B580435FFF756F8A4003F1B380099
:10161000FEF72FFE724B1B78002B02D0009EFFF7C7
:101620001AF82B68019A1C1213406E4A9B009B58B3
:101630000435FFF740F8A4003E1B3000FEF74BFED8
:10164000674B30601B78371D002B02D0009EFFF7E0
:1016500002F82B68019A1C121340624A9B009B58A7
:101660000435FFF728F8A4003F1B3800FEF76AFE98
:101670005B4B1B78002B02D0009EFEF7ECFF2B6823
:10168000019A1C121340574A9B009B580435FFF7E0
:1016900012F8A4003E1B3000FEF78EFE504B306067
:1016A0001B78371D002B02D0009EFEF7D4FF2B685D
:1016B000019A1C1213404B4A9B009B580435FEF7BD
:1016C000FAFF039A3B1D0493454C9B1A8B2B04DDB8
:1016D0001A23009E2370FEF7BEFF01F02BFD0123AD
:1016E0004000184323783860002B03D0009E049FED
:1016F000FEF7B1FF2B68019A1C121340394A9B0078
:101700009B58049F0435FEF7D6FF039A3B1D0493B4
:10171000334C9B1A8B2B04DD1A23009E2370FEF79B
:101720009AFF01F0FDFC304B4000184001231843A4
:1017300023783860002B03D0009E049FFEF78BFFB8
:101740002B68019A1C121340264A9B009B58049F49
:101750000435FEF7B0FFA4003E1B3000FEF776FE16
:101760001F4B30601B78371D002B02D0009EFEF708
:1017700072FF2B68019A1C1213401A4A9B009B5857
:101780000435FEF798FFA4003F1B3800FEF776FEF5
:10179000134B1B78002B02D0009EFEF75CFF2B68DA
:1017A000019A1C1213400F4A9B009B580435FEF708
:1017B00082FF0123A600BE1B20001A003100FEF7A5
:1017C000B1FE0A4C2068643001F04EF8002800D1C8
:1017D000AEE2029B21685A78054801F06EFA1CE0DF
:1017E0004C010020D0650000FEFFFF7F5401002067
:1017F00058010020A600BE1B20000123002231005A
:10180000FEF790FEE34C2068643001F02DF80028CC
:1018100000D18DE2E04801F041F90223029A37003D
:10182000137001F087FC236805331818029B586079
:10183000FEF725FFA4003E1B300001F0ADFCD74BA6
:1018400030601B78371D002B02D0009EFEF703FF8F
:101850002B68019A1C121340D14A9B009B580435F7
:10186000FEF729FFA4003E1B300001F097FCCB4B94
:1018700030601B78371D002B02D0009EFEF7EBFE78
:101880002B68019A1C121340C54A9B009B580435D3
:10189000FEF711FFA4003E1B300001F081FCBF4B9E
:1018A00030601B78371D002B02D0009EFEF7D3FE60
:1018B0002B68019A1C121340B94A9B009B580435AF
:1018C000FEF7F9FEA4003F1B380001F087FCB34B84
:1018D0001B78002B02D0009EFEF7BDFE2B68019AFC
:1018E0001C121340AE4A9B009B580435FEF7E3FEE2
:1018F000A4003E1B300001F093FCA84B30601B7825
:10190000371D002B02D0009EFEF7A5FE2B68019A22
:101910001C121340A24A9B009B580435FEF7CBFED5
:10192000A4003F1B380001F0ADFC9C4B1B78002B42
:1019300002D0009EFEF78FFE2B68019A1C12134006
:10194000974A9B009B580435FEF7B5FE0121200005
:1019500001F080FC914B1B78002B02D0009EFEF71B
:101960007AFE2B68019A1C1213408D4A9B009B58EB
:101970000435FEF7A0FE0021200001F06BFC874B30
:101980001B78002B02D0009EFEF765FE2B68019AA3
:101990001C121340824A9B009B580435FEF78BFEB5
:1019A000A4003E1B300001F08BFC7C4B30601B78A8
:1019B000371D002B02D0009EFEF74DFE2B68019ACA
:1019C0001C121340764A9B009B580435FEF773FEA9
:1019D000A4003E1B300001F087FC704B30601B7888
:1019E000371D002B02D0009EFEF735FE2B68019AB2
:1019F0001C1213406A4A9B009B580435FEF75BFE9D
:101A0000A4003F1B380001F049FC644B1B78002BFD
:101A100002D0009EFEF71FFE2B68019A1C12134095
:101A20005F4A9B009B580435FEF745FEA4003F1B10
:101A3000380002F013F9594B1B78002B02D0009E9E
:101A4000FEF709FE2B68019A1C121340544A9B00B2
:101A50009B580435FEF72FFEA4003E1B300002F019
:101A60004FF94E4B30601B78371D002B02D0009E83
:101A7000FEF7F1FD2B68019A1C121340484A9B00A7
:101A80009B580435FEF717FEA4003F1B380002F0F8
:101A900083F8424B1B78002B02D0009EFEF7DBFD43
:101AA0002B68019A1C1213403D4A9B009B58043539
:101AB000FEF701FEA4003E1B300002F083F8374B16
:101AC00030601B78371D002B02D0009EFEF7C3FD4F
:101AD0002B68019A1C121340314A9B009B58043515
:101AE000FEF7E9FDA4003F1B380001F0EFFE2B4B91
:101AF0001B78002B02D0009EFEF7ADFD2B68019AEB
:101B00001C121340264A9B009B580435FEF7D3FD58
:101B1000A4003F1B380001F0E5FE204B1B78002B92
:101B200002D0009EFEF797FD2B68019A1C1213400D
:101B30001B4A9B009B580435FEF7BDFDA4003F1BCC
:101B4000380001F0D5FE154B1B78002B02D0009E0B
:101B5000FEF781FD2B68019A1C121340104A9B006E
:101B60009B580435FEF7A7FDA4003F1B380001F089
:101B7000DBFE0A4B1B78002B02D0009EFEF76BFDAC
:101B80002B68019A1C121340054A9B009B58043590
:101B9000FEF791FD54010020580100204C01002067
:101BA000D0650000A4003E1B300002F033F99F4BCB
:101BB00030601B78371D002B02D0009EFEF74BFDD6
:101BC0002B68019A1C121340994A9B009B580435BC
:101BD000FEF771FDA4003E1B300002F023F9934B89
:101BE00030601B78371D002B02D0009EFEF733FDBE
:101BF0002B68019A1C1213408D4A9B009B58043598
:101C0000FEF759FDA4003E1B300002F013F9874B8C
:101C100030601B78371D002B02D0009EFEF71BFDA5
:101C20002B68019A1C121340814A9B009B58043573
:101C3000FEF741FDA4003E1B300001F0D1FF7B4BBD
:101C400030601B78371D002B02D0009EFEF703FD8D
:101C50002B68019A1C121340754A9B009B5804354F
:101C6000FEF729FDA4003F1B380001F079FE6F4B01
:101C70001B78002B02D0009EFEF7EDFC2B68019A2A
:101C80001C1213406A4A9B009B580435FEF713FD53
:101C9000A300FF1A3900200001F014FF634B1B78EA
:101CA000002B02D0009EFEF7D6FC2B68019A1C1276
:101CB00013405F4A9B009B580435FEF7FCFCA400D0
:101CC0003E1B300001F0CAFE584B30601B78371DB8
:101CD000002B02D0009EFEF7BEFC2B68019A1C125E
:101CE0001340534A9B009B580435FEF7E4FCA300C5
:101CF000FF1A3900200001F093FE4C4B1B78002B9B
:101D000002D0009EFEF7A7FC2B68019A1C1213401C
:101D1000474A9B009B580435FEF7CDFCA4003B1BB3
:101D20001800049301F05FFB01F05BFB002802D177
:101D3000043DFEF7A4FC3D4B1B78002B03D0009E16
:101D4000049FFEF788FC2B68019A1C121340384A46
:101D50009B009B58049F0435FEF7ADFCA300FE1AC0
:101D600020003100049301F037FB049B3060FC1A23
:101D70002E4B271D1B78002B02D0009EFEF76BFC1C
:101D80002B68019A1C121340294A9B009B5804356A
:101D9000FEF791FCA300FF1A3900200001F028FB98
:101DA000224B1B78002B02D0009EFEF754FC2B68C0
:101DB000019A1C1213401E4A9B009B580435FEF7E3
:101DC0007AFCA300FF1A3900200000F0D7FC174B63
:101DD0001B78002B02D0009EFEF73DFC2B68019A79
:101DE0001C121340124A9B009B580435FEF763FCFB
:101DF000A300FE1A20003100049300F0BFFC049BF6
:101E00003060FC1A094B271D1B78002B02D0009E66
:101E1000FEF721FC2B68019A1C121340044A9B0018
:101E20009B580435FEF747FC07B0F0BD4C0100207D
:101E3000D0650000014B1870002070474C01002055
:101E4000F0B50023A02787B05A1E0492002B05DCB2
:101E500001F0EEFB00F056FF1923049300250395D3
:101E60000295254B19688D4201DB049BECE7234B5F
:101E70001A680132914200DC00221A601B68204E71
:101E800001937B439A199B5D05923400032B01D18A
:101E900010002CE0002B2DD0012B0CD1029B002B2D
:101EA00002D101F03DF90290019A02997A43A418F7
:101EB0006368CB1A0FE0022B12D1039B002B02D1D7
:101EC00001F038F90390019A03997A43A4186368E2
:101ED000CB1A9B029B0A0B498B4201D80323B354B4
:101EE000019B074A7B439B5C032B03D10598FEF7BC
:101EF0008BFBBAE70135B4E7500100200000002059
:101F0000381000209F860100054B01211A68054BFF
:101F10001A600023044AD1500433642BFBD170476C
:101F20008004002078040020701E002000B59BB0C3
:101F30000200054901A803F08DFC01A800F0AEFDE8
:101F400000F0E0FEFCE7C046D067000037B5174D53
:101F500004002868002801D003F070F8A4002000D5
:101F600003F062F82860002801D1114809E001ABB4
:101F7000984208D20F4B02196B440193934202D24C
:101F80000D48FFF7D3FF042802D808302860083C2A
:101F90002B680A4A1C191360094B01211C6000239D
:101FA000084AD1500433642BFBD137BD8004002094
:101FB000E16700001CFCFFFF1168000078040020AE
:101FC0007C040020701E002070B50D4D0D4E2B6856
:101FD0004C1CA40036681C19B44203D90A20FFF730
:101FE00029FF0BE02C601D00AC4201D904C5FBE7C2
:101FF0000F220901104008431860180070BDC04648
:10200000780400207C0400200322CB1C70B50C0057
:10201000D9171140C9180500891000220420FFF7C4
:10202000D3FF0023A34204DAE95CC2181171013323
:10203000F8E7E1430023C917214041180B7170BD37
:1020400010B5830706D1042804D90F2304C8134010
:10205000042B03D00E20FFF7EDFE014810BDC04653
:102060001869000030B502248025094B094AED00AB
:102070009C505C59002CFCD0A124E400884204D27E
:102080008025ED0018514019F8E70021995030BD26
:1020900000E001400405000010B5002804D19020A4
:1020A00092210002890203E0922080218002C9026D
:1020B000FFF7D8FF10BD002802D092239B0201E059
:1020C00090231B021B6800201A0E532A01D11B0209
:1020D000180A704730B501248025064A064BED00EA
:1020E000D4505459002CFCD001600021014AD15039
:1020F00030BDC04600E001400405000010B50028D6
:1021000002D09220800201E090200002A623090262
:10211000DB05090A1943FFF7DDFF10BDF0B5012407
:10212000802503000F4F08000F49ED007C507C59BB
:10213000002CFCD09C46002810DD5478167893784B
:10214000240234431B0423431C00D37801381B06AC
:102150002343644608C40432A446ECE700237B50C2
:10216000F0BDC04600E001400405000070B5050068
:102170004B680A009C1C2100FFF7D0FFA000281824
:1021800070BD0000154B1B68002B04D080219223EA
:10219000C9029B0203E09221902389021B020028BE
:1021A00007D1191D5B6802001B0E522B14D10A00C7
:1021B00012E0002281420FD903681B0E522B0BD173
:1021C000436802339B00C318994205D91A68110E5F
:1021D0000022522900D11A00100070478406002006
:1021E0008022F0B5520085B00021624802F039FF2C
:1021F000802200215200604802F033FF5F4B1B68D1
:102200001A00029353425A4110000392FFF744FF11
:10221000029B002B01D15A4C00E05A4C0020FFF7E2
:10222000B1FFFF270500002D00D194E02B681A12A2
:102230001B143A403B4001921A000A3A092A43D83B
:102240004C4B019A995C002900D07FE010224E4847
:1022500002F007FF2E00336801991A123A409142AA
:1022600017D11A143A400B2A06D0132A0CD00A2A86
:102270000FD1454B1E600CE03B40022B09DC424A6B
:102280009B00D3185E6004E0102200213E4802F05B
:10229000E8FE3000FFF776FF061EDCD13A4B1968E6
:1022A00000290FD02000FFF761FF0400374E31688E
:1022B000002903D02000FFF759FF0400344B0436F7
:1022C000B342F4D12B4B3EE0143B092B3ED82A4BB2
:1022D000019A995C002939D108222E4802F0C1FEEA
:1022E0002E0033681A143A40152A0BD01D2A11D03B
:1022F000142A14D1019A1B123B409A420FD1254B4C
:102300001E600CE0019A1B123B409A4207D1214B00
:102310005E6004E0082200211E4802F0A2FE3000A8
:10232000FFF730FF061EDCD11A4E3168002909D0B4
:102330002000FFF71BFF71680400002902D0FFF79F
:1023400015FF04000C4B0121019A99542800FFF756
:1023500019FF050067E70298FFF7ADFE411C0398DF
:10236000FFF7CCFE054B039A1A600B4B1C6005B0BF
:10237000F0BDC046840500208404002084060020AF
:102380000448020004900000D41E0020D81E002043
:10239000E41E0020E41E00208806002070B5002006
:1023A000FFF789FE04000120FFF785FE844200DA72
:1023B00004000A4B1E687542754128001D60FFF736
:1023C0006BFE002E01D0064B00E0064B064A2800AB
:1023D000611C1360FFF792FE70BDC04684060020AA
:1023E000049000000448020088060020F8B5002090
:1023F000FFF761FE07000120FFF75DFE3E00224D62
:102400000643224C0CD180219020C9020002FFF724
:1024100029FE01213000FFF771FE2E601C4B2FE0DA
:10242000874208DD002392212B60194B890223602B
:102430002368002011E0012380212B60154BC90285
:102440002360F5E71A68551C18D0120E522A07D1DE
:1024500001205A68023292009B188B42F2D311E09D
:10246000002800D023600C4C0C49200003F01EFA19
:10247000200000F065FEFFF791FF04E0002802D085
:10248000236000E02160F8BD84060020880600205B
:102490000490000004480200EC1E0020896800003F
:1024A000F0B585B0039203220333DC171440294EA4
:1024B000E3189C10336801900291002B02D0802217
:1024C000D20201E092229202234FA51C3B68AD008C
:1024D0005B199A4217D2FFF783FE3368002B02D0B4
:1024E0008022D20201E0922292023B685B199A425A
:1024F00009D21A4C1A49200003F0D8F9200000F044
:102500001FFE002023E0029B3E681B06190C6B4651
:102510001A7BA423DB051343019A0B431104FF220A
:102520001204114019433000FFF7D4FD3300301D71
:10253000083321000193FFF7CDFD01980A9A21008D
:10254000FFF7ECFD3000019B083D5D193D6005B0D3
:10255000F0BDC0468406002088060020EC1E002046
:10256000B268000070B59AB0FFF740FFFF221F4C21
:10257000D2000021200002F074FD0020FFF702FECF
:10258000FF25002600281AD003681A142A400A2AB8
:1025900008D11A122A40FF2A0ED0D200A1180B71BE
:1025A000A05009E0132A07D11B122B40FF2B03D0A8
:1025B000DB00E2181671E650FFF7E4FDE2E7FF21C9
:1025C0000200C900235808305D1EAB41D218884272
:1025D000F8D1074901A803F03DF901A800F05EFA1F
:1025E000044800F05BFA1AB070BDC04678160020AF
:1025F000D9680000F1680000044A05491368C8540E
:1026000001339B059B0D13607047C0468C0A002068
:102610008C060020114A70B51368114C984211DAEB
:10262000015D451CFA39012906D8AB4206DD2118A7
:10263000497801391F2901D92800EFE70100251A3F
:10264000461C02D10023136006E0665C6E54013123
:102650008B42FADC181A106070BDC046900A002048
:10266000980A002010B500F05BFD064B1A689042F6
:1026700001D200221A601B68C01A034B83428041BA
:10268000404210BD940A0020204E000010B5094AB7
:10269000094C1268236893420AD0084AD05C00F0C3
:1026A00079FE002804D0236801339B059B0D23602D
:1026B00010BDC0468C0A0020980E00208C06002019
:1026C00010B50400064B074A1B6812689B1ADB43CF
:1026D0009B059B0DA34202DAFFF7D8FFF2E710BD7E
:1026E0008C0A0020980E0020F7B506000191151EF7
:1026F0002FD05768B800441C0630FFF7E1FFFB20DD
:10270000FFF77AFF1C20FFF777FFF0B2FFF774FFA7
:10271000E0B22412FFF770FFE0B2FFF76DFF6B46E7
:102720001879FFF769FF0026BE4212DAB300EB18F2
:102730009C680136E0B2FFF75FFF2012C0B2FFF7DE
:102740005BFF2014C0B2FFF757FF200EFFF754FFC6
:10275000EAE7F7BD70B5074D2C68042C08DC0C23A4
:102760006343054E01349851F31859609A602C6008
:1027700070BDC0469C0E0020501F0020F0B589B0EF
:1027800004900E0001284BDD284B08680293830754
:1027900009D1042807D90F2302681340042B02D162
:1027A000FFF74EFC0290214B70680393830709D119
:1027B000042807D90F2302681340042B02D1FFF726
:1027C0003FFC039000271A4B1A4D1B680593059B8D
:1027D0009F4225DA2B1F0299186803F05DF8002844
:1027E0001BD12B686C6806930190019B069A93425B
:1027F00013DA20680399079403F04EF80834002890
:1028000007D131000498079B08315B68023898476C
:1028100009E0019B01330193E7E701370C35D6E767
:102820001B20FFF707FB09B0F0BDC0461869000088
:102830009C0E0020541F002010B501F089F900F013
:1028400069FD00F0DBFD10BDC82210B5D2000021EB
:10285000034802F006FC0022024B1A6010BDC0467D
:102860003810002050010020064B074A1B681268F0
:102870009B1ADB439B059B0D0122834200DC002257
:10288000100070478C0A0020980E0020F8B5050053
:102890000C0016001F1E0ED10320FFF7E5FF0028D5
:1028A00027D0FA20FFF7A8FEE8B2FFF7A5FEE0B2B6
:1028B000FFF7A2FE1DE0501DFFF7D6FF002818D03D
:1028C000FB20FFF799FEE8B2FFF796FEE0B2FFF7B4
:1028D00093FEF0B2FFF790FE3012C0B2FFF78CFE0D
:1028E0003C00E31B9E4204DD2078FFF785FE0134A7
:1028F000F7E7F8BD70B50024A0250B4B1B689C4280
:102900000EDA2A006243094BD3181A78002A05D040
:102910005978002311201A00FFF7B8FF0134ECE7C3
:10292000FFF792FF70BDC046500100203810002014
:102930000123F3B50400FFB00D0010001A420DD0C2
:1029400002AA1370431002A9537042121B0E4014C6
:102950008A700B71C8700B00052273E003231340CB
:102960001ED1042A1CD90F2201680A40042A17D15B
:10297000023302AA1370FFF763FB060002F09EFF0A
:10298000F823FF33984200DD18000023834205DA64
:1029900001335A1EB25C02A9CA54F7E7421C50E048
:1029A000042801D0002809D1032302AA0438137097
:1029B0004342434153701300022243E0002B45D1B0
:1029C000042843D90F2102681140052912D104338C
:1029D00002A90B70F8231209FF3392009A4200DD1E
:1029E0001A00002393422BDA0133C118C97802AED2
:1029F000F154F7E7062929D101390E00120956438F
:102A00000196F826019FFF36B7421FDC02AE3170F7
:102A10000136934213DA01270133990041583942B4
:102A200001D0394100E00A49012737700F12717057
:102A3000B7700F14090EF77031710536E9E7019A86
:102A4000013202AB29002000FFF720FF7FB0F3BD69
:102A500019FCFFFF70B5A023050000240D4A1800E3
:102A6000604380184178A94203D001340A2CF6D182
:102A70000FE0A022002102F0F4FA074A1368013B9C
:102A8000A34200D11460002329001A001120FFF78F
:102A9000FDFE70BD381000205001002010B5B2B00E
:102AA00002236A460400137002F008FFC72800DD05
:102AB000C7200023834205DA694601335A1EA25C0F
:102AC000CA54F7E7421C6B46FF211420FFF7DEFED5
:102AD00032B010BDF7B5234B06001B68A020009351
:102AE00000232149009A93420ADA02005A438A18C5
:102AF0005478B44202D11278002A32D10133F1E77E
:102B00000024A0231A00624301920199164A551825
:102B10002F78002F06D001340A2CF3D11348FFF789
:102B2000BDFF1EE0A0223900280002F09AFA03231C
:102B30000D4A01996E7053540D4BF200D358AE708C
:102B4000AB600223EB60009B2F616F61A34202DC4C
:102B5000044B01341C60002331001A001020FFF7E1
:102B600095FEF7BD5001002038100020AC69000030
:102B70007816002010B5FFF7BDFE0024064BE200DA
:102B8000D3181B79043B012B02D8E0B2FFF7A2FF58
:102B90000134FF2CF2D110BD78160020F7B50E00DD
:102BA00000247F250190194BE200D11809790629EC
:102BB00001D0032926D1985883682B401C2B21D1A2
:102BC000C3681A002A40042A1CD102692A40192A23
:102BD00018D11B0A01339B000C30C018FFF730FAE4
:102BE000070002F06BFE0023B0420BD19E4206DDCF
:102BF000019AF95CD25C914204D10133F6E7E0B26C
:102C0000FFF768FF0134FF2CCDD1F7BD7816002007
:102C100037B500240500FFF76DFE01A8019400F010
:102C20003DFB200000F05EFE00F002FD00F070FBB6
:102C300000F06FFB00F00CFF00F09CFA0548FFF776
:102C40002DFFA54204D0FFF75FF90348FFF726FFE9
:102C500037BDC046C1690000D9690000002310B526
:102C600001001A001120FFF711FE10BD07B56B46D9
:102C7000197069465A7013128B701314120ECB70B0
:102C80000A716B46010005221320FFF7FFFD07BD07
:102C900010B50A0001001220FFF74AFE10BD70B502
:102CA000050008000C003230FFF70AFD2B0022005F
:102CB00000211B20FFF7EAFD70BD10B50C000300DA
:102CC000110014202200FFF7E1FD10BD70B50600D1
:102CD0000020FFF757FA0024FF25002810D00368D2
:102CE0001A142A40152A05D11B122B40B34204D1D5
:102CF000040002E01D2A00D10024FFF743FAECE7AC
:102D0000200070BDF0B580279DB0FFF7BFFCB94D26
:102D1000B94C2868FF00391A201800F021FB2B68F5
:102D20000600C3182B60002B00D1DBE1002E0DDD67
:102D30002868391A201800F013FB2B6806001B18AE
:102D40002B6000F0EDF9AD4B1860EFE72378FA2B1C
:102D500000D00CE12B68022B06DCFFF783FC002877
:102D600000D1BFE10120B8E16078A57802381828C9
:102D700000D9FAE001F040FF0D1E22262932F93D6C
:102D8000676F7589DAEFF9F9F9F9F9F9F9F9F9F9EC
:102D9000F300FF2D00D1E8E02800FFF75BFE0022E2
:102DA0009749EB005A50CB181A7129000092130072
:102DB00013204DE02800FFF78DFED6E02800FFF736
:102DC00049FED2E0FFF7D6FECFE0FFF793FD0020EB
:102DD000FFF71EFF8B48FFF761FEC6E0182D00D9F4
:102DE000C3E0894BAA00D25829001520FFF7A0FDA7
:102DF000BBE000242000FFF769FF071E03D1013468
:102E0000192CF7D1B1E0083002F058FD060005306A
:102E1000FFF756FCFB20FFF7EFFB1D20FFF7ECFB55
:102E2000E0B2FFF7E9FBF0B2FFF7E6FB3012C0B209
:102E3000FFF7E2FB0025AE42E1DD7B19187AFFF7D0
:102E4000DBFB0135F7E700211D200B000A00009194
:102E5000FFF726FB89E000222900009213002720BB
:102E6000F6E700F075F903AC684A64210090684BFE
:102E7000200002F0BDFC02232000237002F01EFDA2
:102E800023000200002116206DE000245C4AE300CC
:102E9000D558002D46D06B689E00701DFFF710FCC2
:102EA0002B0000253200083321000120FFF7EEFC43
:102EB0000020FFF767F92E002F0000281DD0FF210A
:102EC00003681A120A40A24214D11A140A400B2AAB
:102ED00007D10B400DD0012B09D0022B00D1FFE010
:102EE00008E0132A06D100252E002F0002E006007C
:102EF00000E00700FFF746F9DFE7002E04D03200BC
:102F000001212000FFF7F0FB002D04D02A00022150
:102F10002000FFF7E9FB002F04D03A000021200039
:102F2000FFF7E2FB0134FF2CB0D11EE0FFF7E2FC1B
:102F300000250024290000942300220013200135DD
:102F4000FFF7AEFAFF2DF4D1FF222100D2002C486A
:102F500002F087F809E00120FFF75AFE05E00023A0
:102F60001A201A001900FFF791FC0320B5E0FB2B93
:102F700000D0F7E62A68042A00DCEEE62679E0783D
:102F8000244B360206439E4200DDEBE6331D9A4297
:102F900000DCE2E6E35CFE2B00D0E3E66078A57897
:102FA000731E1C2868D007D8082835D01B285ED08F
:102FB000012800D090E007E01E2800D17EE066D313
:102FC0001F2800D180E087E0FF2D00D184E0280099
:102FD000FFF740FD67790634B31E290000943A00DC
:102FE0000A20FFF75DFA064BED00E8505D192F71DE
:102FF00072E0C046900A0020980A0020940A00203F
:1030000078160020E9690000701E0020006A0000A8
:10301000FB690000F6030000182D5DD860790228D6
:1030200013D003281BD0012856D1A71D7A78A47984
:10303000BB78120222431B0413431A00FB78AD0035
:103040001B0613435B0003430EE0002B44DDB11E5F
:10305000A01DFEF7D9FF244BAD00E8503CE0A3795A
:10306000AD005A1E93419B001F4AAB5034E0601DD7
:103070001900FFF793FD2FE0FF2D2DD06279022A72
:103080002AD80634B31E009429000B2022E0632BBB
:1030900000DD6323002203A8934204DDA1184979CF
:1030A00081540132F7E7D9430022C917194041186A
:1030B0000A7001330090290015200BE005340094BC
:1030C000002229001E2005E0042B05D10022290042
:1030D00005340094FFF7E4F9701DFFF79BFA01E057
:1030E000050007E71DB0F0BD701E002000207047EE
:1030F0000020704700207047002070470122002008
:10310000054B06491A615850033004315850801855
:10311000083158501A6070470080004004050000D4
:103120000122034B1A64A822D20098587047C04667
:103130000080004010B5FFF7F3FF800A10BD0000CB
:1031400010B50100014801F00BFB10BDC40F0020B9
:1031500000487047106A000070B5054E0400335CEB
:103160000D008B4202D001F023FA355570BDC046E8
:10317000A00E002070B50024064D635D012B05D123
:103180000021200001F014FA0023635501341D2CA6
:10319000F2D170BDA00E00200D2070473B2070477B
:1031A000036870B55B100120052B12D8094A9B00FB
:1031B0009C58094D2B5D002B05D00021200001F00B
:1031C000F7F900232B55200001F09CF80123400063
:1031D000184370BD406A0000A00E002070B503685F
:1031E00045685C106D1004D40B4B9D4202DD1D0040
:1031F00000E000251C2C0DD8084E335D012B05D0B6
:103200000121200001F0D4F90123335529002000C9
:1032100001F006F970BDC046FF030000A00E0020BB
:1032200070B5046864101C2C0FD8094D2B5D002B61
:1032300005D00021200001F0BBF900232B55200010
:1032400001F0EAF90423012800D00023180070BD22
:10325000A00E002070B504000D001C280ED8084EEA
:10326000335C012B04D0012101F0A2F90123335575
:10327000290020004D1EA94101F0B8F970BDC046DB
:10328000A00E0020436810B5191F4A424A41006849
:1032900011004010FFF7DEFF10BD000037B5694692
:1032A0000200064B684630CB30C11368042B02D1B4
:1032B00000F01EFB01E000F037FB37BD086A00009C
:1032C00010B5084C6379002B05D00021052001F0D2
:1032D0006FF900236371052001F09EF943425841C4
:1032E000800010BDA00E002010B5084CE37A002B22
:1032F00005D000210B2001F05BF90023E3720B20C5
:1033000001F08AF943425841800010BDA00E002010
:103310007047704710B5034A04210348FFF71AFAB3
:1033200010BDC046040000201A6A0000E12110B55B
:103330004902094801F05BFAFFF7E0FE0A2000F0BD
:10334000DBFF0023FF21054A995401331D2BFBD1DC
:1033500000F07EFB10BDC046C40F0020A00E002070
:10336000F8B50B4E070030000D0001F07FFA041E87
:10337000AC4200DD2C003D00EB1B9C4205DD300023
:1033800001F07EFA28700135F6E72000F8BDC0464E
:10339000C40F002010B50100014801F02FFA10BD44
:1033A000C40F002010B51D20FEF744FD10BD10B560
:1033B0001D20FEF73FFD10BD10B51D20FEF73AFDA4
:1033C000002010BD10B51D20FEF734FD10BD10B556
:1033D0001D20FEF72FFD10BD10B51D20FEF72AFDA4
:1033E00010BD0420704710B51D20FEF723FD10BD51
:1033F00010B51D20FEF71EFD10BD000010B5034ADC
:1034000006210348FFF7A6F910BDC046240000209E
:10341000586A00000123034A1360034A1068984069
:1034200018437047C80E0020D00E0020202800D975
:103430000020084B8000C25801239340064A0749E8
:103440001360074A1160074A07491160074A136071
:103450007047C046946E0000C40E0020080500505E
:10346000E00E0020D80E00200C050050180500507A
:10347000F0B5EFF310810123194083F31088134E48
:10348000134AB4461268013A9340124A1468124A29
:103490001568124A002B15D0166803420BD026601F
:1034A000C046C046C046C046C046C046C046C046EC
:1034B00016682E6004E067463E601668084F3E605E
:1034C0005B08E7E781F31088F0BDC04608050050AF
:1034D0005C000020E00E0020D80E0020C40E00206A
:1034E0000C05005030B585B001AD0C22064928000E
:1034F00001F0AEFD0024285D01210134FFF72CFE10
:103500000C2CF8D105B030BDC26A0000F7B53C4CB8
:103510000322210068460C3101F09AFD21000322AC
:103520000F3101A801F094FDFFF704FE354B364C36
:10353000C0182368984201D2002323602568002D1B
:1035400036D12E006B469F5D01213800FFF704FE47
:1035500001360021380001F049F8032EF2D100278E
:103560006B460433DE5D01213000FFF7F5FD3000CE
:10357000012101F03BF832200138C046C046C04668
:10358000C046C046C046C046C046C046C046C0460B
:10359000C046F1D16B460433D85D00210137FFF7F7
:1035A000DBFD032FDCD1FFF7C5FD0530206024E0F3
:1035B000FFF7C0FD002723683D0098421DD3134E3E
:1035C00037606B460433D85D00F09CFE33680137EA
:1035D000C0183060032FF4D10D4B181A01D430609D
:1035E00001E0002333603068052101F099FB0023DE
:1035F0000125084A3060236013602800FEBDC046E4
:10360000C26A000010270000C00E0020D00E00206B
:103610008F020000C80E002010B50124044001D024
:10362000441002E00D20FEF705FC200010BD000054
:103630007FB5A14E3368002B06D1A04A1268002A3C
:1036400002D1FFF763FF36E19D4D2A68002A2AD197
:103650009C4A1268002A07D0FFF758FF002800D1C3
:1036600029E1FFF73FFF05E0944A1268002A01D1E3
:10367000002BF6D1914B19681A00002911D034683B
:10368000002C0ED101AD0C228F4928001C6001F0E6
:10369000DFFC285D00210134FFF75EFD0C2CF8D122
:1036A00009E13368136000211A2000F09FFF002118
:1036B0001B2000F09BFF00211C2000F097FF2E68CC
:1036C000012E56D0022E00D19CE0002E00D0ECE05E
:1036D00001363100794C03202368994300F086FFBE
:1036E0000420216801400B005942594100F07EFF3F
:1036F000102123680A200B405942594100F076FFFF
:103700008021236809010B4059425941062000F0ED
:103710006DFF8021236809020B405942594107205F
:1037200000F064FF8021236849020B40594259414F
:10373000092000F05BFF8021236889020B40594279
:103740005941192000F052FF80212368C9020B4023
:1037500059425941182000F049FF802321681B037A
:103760000B4059425941172000F040FF31001A2008
:1037700099E00221514C172023680B4059425941CE
:1037800000F034FF0821236818200B4059425941AA
:1037900000F02CFF80212368C9000B405942594199
:1037A000042000F023FF8021236849010B40594287
:1037B00059410A2000F01AFF80212368C9010B40FB
:1037C00059425941032000F011FF802123688903E9
:1037D0000B4059425941092000F008FF802321681D
:1037E0001B040B4059425941192000F0FFFE3100E3
:1037F000062000F0FBFE3100072000F0F7FE31004C
:103800001B2050E020212D4C172023680B405942EB
:10381000594100F0EBFE4021236818200B4059422B
:10382000594100F0E3FE8021236819200B405942E2
:10383000594100F0DBFE8021236849000B405942CA
:103840005941092000F0D2FE8021236889000B40F5
:1038500059425941072000F0C9FE8021236889019F
:103860000B4059425941062000F0C0FE80212368D8
:1038700049030B40594259410A2000F0B7FE80210C
:103880002368C9030B4059425941032000F0AEFEA2
:10389000802321685B040B4059425941042000F009
:1038A000A5FE01211C2000F0A1FE2B680321581C5D
:1038B00001F01CFB29607FBDD40E0020CC0E00203F
:1038C000DC0E0020C80E0020C26A0000006810B59F
:1038D000C30703D5FFF7A0FE014B186010BDC0461B
:1038E000D40E00200022014B1A607047D40E002035
:1038F00070B505000068FFF78FFE04006868FFF7E9
:103900008BFE631E042B0CD80138042809D805222D
:103910005043043AC3189A40130002490A681343FB
:103920000B6070BDD40E002070B505000068FFF775
:1039300073FE04006868FFF76FFE631E042B0CD84B
:103940000138042809D805225043043AC3189A4084
:10395000130002490A689A430A6070BDD40E002021
:103960002C4BF7B51B680400002B03D1012040420B
:10397000FFF75CFD01262468344219D0FF22631052
:10398000180212041040FF22611212020A40DBB238
:1039900010431843204B1B68202B06D1B4401F4B0B
:1039A000A40EA400E35800021843FFF761FD30E0C5
:1039B000032525402DD1042C2BD90F232268134039
:1039C000062B26D1FF27130901933F04019B9D423B
:1039D0001FDAAB00E3185A68324218D053101802AD
:1039E0003840FF2184460902501208406146DBB28C
:1039F00008431843084B1B68202B06D15200920E37
:103A0000064B9200D35800021843FFF731FD0135F1
:103A1000DCE7F7BDE00E00205C000020E86A000053
:103A20000B6810B50200D80701D5581001E001203D
:103A300040421823012A03DD4A68042A00D10833D2
:103A4000024A1360FFF7F2FC10BDC0465C00002084
:103A5000012010B54042FFF7E9FC10BD0068F8B541
:103A6000C30702D5FFF7D8FD0BE0830726D1042852
:103A700024D90F2203681A40042A1FD11B091DD024
:103A800000790300203B5E2B18D805220020534309
:103A90000B4E9D18043AAB420CD0052110249F5DBB
:103AA0003C4200D080180139520064100029F7D13F
:103AB0000133F0E701234000184300E00120F8BD86
:103AC000E86B0000F0B5040085B008680E00FFF751
:103AD000A3FD0190022C07DD7068FFF79DFD040037
:103AE000B068FFF799FD01E001200400174B011DAC
:103AF0001A680523461E434301200027844602918D
:103B0000211D053B039102998E4219D0611E039D30
:103B1000A94212D0042E0DD804290BD8019D5F189C
:103B2000054203D06546BD402A4302E06546BD40DC
:103B3000AA43012740000131E9E701360533E2E7F6
:103B4000002F01D0014B1A6005B0F0BDD40E00204B
:103B500010B5034A01210348FEF7FCFD10BDC04625
:103B600054000020D46A000010B501210D20FFF799
:103B7000F3FA01210E20FFF7EFFA00210F20FFF7E3
:103B8000EBFA044C200000F0C3F91021200000F0F3
:103B9000DBF910BDF40E002010B504680D20E3071A
:103BA00003D56410FF2C03D91720FEF743F906E074
:103BB000FFF7DAFFE1B2024800F0E8F9002010BD9B
:103BC000F40E002010B5FFF7CFFF0021034800F0EE
:103BD000DDF901234000184310BDC046F40E00205B
:103BE0000122094B1A60094A1368002BFCD00322FA
:103BF000074B1B68D8171040C018012380100638E7
:103C0000400018437047C04600C0004000C100405B
:103C100008C50040F7B50F4F06003B680D00019244
:103C20000D4C002B04D1200000F036FA01233B603C
:103C3000F1B2200000F0BEFAE9B2200000F0EDF988
:103C40006B462000197900F0E8F9200000F01CFB19
:103C5000F7BDC046E40E0020080F002010B5012477
:103C60000368234205D04168214202D08268224283
:103C700001D10D2004E058104910802803D91520E7
:103C8000FEF7D8F80BE0FF2901D91620F8E752100B
:103C9000FF2A01D91720F3E7FFF7BCFF002010BD72
:103CA000F8B5154F05003B680E00144C002B04D1ED
:103CB000200000F0F1F901233B60EDB22900200063
:103CC00000F078FAF1B2200000F0A7F900212000FE
:103CD00000F07CFA002801D040420CE001222900CB
:103CE000200000F062FA200000F08DF90028FAD0E0
:103CF000200000F08DF9F8BDE40E0020080F002030
:103D000010B501240368234202D04168214201D149
:103D10000D2004E058104910802803D91520FEF723
:103D200089F807E0FF2901D91620F8E7FFF7B8FF67
:103D30004000204310BD0000002370B5344D040046
:103D4000EB5601332BD10D211D20FFF7A9FF5A2877
:103D500004D101222A212A703D380AE00F211920BE
:103D6000FFF79EFF332807D102235F2220212B700B
:103D70001A38FFF74FFF12E00D211E20FFF790FFCA
:103D8000C7280AD1032300222A21A9382B70FFF764
:103D900041FF1B222A211E20EBE700232B7000236A
:103DA000EB56022B06D0032B13D0012B26D121007A
:103DB0001D2010E0012C04D129211920FFF770FFEC
:103DC0000DE0032C15D12B211920FFF769FF043CCE
:103DD00005E021001E200124FFF762FF64427F28D6
:103DE00001DD0138FF3803007F330ADA7F204042CB
:103DF00007E0052C02D12D211920ECE70124002039
:103E0000644264237F21584300F08AFF604370BD01
:103E10006000002010B50120FFF78EFF0123400055
:103E2000184310BD10B50320FFF786FF01234000A3
:103E3000184310BD10B50520FFF77EFF0123400099
:103E4000184310BD10B5FFF771FAE120C000FEF76E
:103E50007DF8FEF7F1FC0448FEF720FEFEF782FB3A
:103E6000FEF788FE10BDC046C169000010B5FDF721
:103E7000E7FF10BD70B5002504AC24780573A94296
:103E800005D10A4B0A4A23210A4801F061F8016072
:103E90000949920052589B0002715B588371A3003C
:103EA0005B58856043710223C37170BD006E0000D2
:103EB000C36D00000E6E0000946E0000037B002BAB
:103EC00004D14373837303610133037370470000AC
:103ED0001FB50191A02100240068C900D2B244504E
:103EE000012A07D0A24203D0032A05D1042202E00E
:103EF000022200E006221343034A8350034B019A37
:103F0000C250012343501FBD54050000240500008A
:103F100010B50400FFF7D2FFA1222368A179D200D7
:103F200099506179064A20009950217904329950BC
:103F3000044B19685A689B68FFF7CAFF10BDC0465A
:103F40000C050000E80E00204BB2002B0CDB802398
:103F50003F290CD81F290CD80F290CD807290CD8B9
:103F600003290CD81B060BE080239B0408E0DB042C
:103F700006E01B0504E05B0502E09B0500E0DB05B5
:103F80000168014A8B507047240500000368074A06
:103F900099501A00FC32D1680029FCD0A321C90035
:103FA00058580023C0B2D3607047C0461C050000BB
:103FB00007B58022074BD2051A6000229A600232B0
:103FC0001A710F230C3200930349023B0348FFF799
:103FD00051FF07BDE80E002000300040F40E002025
:103FE000F8B505000E0017000024BC4208D02B686D
:103FF000315D1B6828009847002801D00134F4E7A0
:104000002000F8BD704710B51C3000F0D5FB10BD86
:1040100010B51C3000F0C2FB10BD70B5437E0D0022
:10402000002B05D06430040000F0D5FB002801D03F
:10403000002004E02000290000F0A1FB012070BD59
:1040400010B51C3000F0BEFB10BD0000F7B50193A9
:10405000FA23002504009B0083600D4B4560083364
:1040600003601C300F00160000F07EFB200064305F
:1040700000F07AFB074AB600B35827616375019BCD
:1040800020009B009B586576A576A375FEBDC046B3
:10409000746E0000946E00000123A022C375837D1E
:1040A0000C49C133FF33D2059B009950437DC13386
:1040B000FF339B009950CC210369074A490499506A
:1040C0000521243A9950817D08329950417D034A57
:1040D000995070470C060000240500000C050000F4
:1040E000F7B5050000200C00019382425CD0161E3B
:1040F000402E00D940262F001C37380000F04AFB24
:10410000B1222B69D20080219C50012289005A5093
:10411000A97E002901D11A621A600024731E2A693F
:10412000A34206D1019B002B03D0802302219B00D8
:10413000D150012313621300FC33D968002902D146
:10414000996A0029F9D0996A00290AD1D960A32374
:10415000DB00D1583800C9B2013400F010FBA64290
:10416000DCD8019A2B69002A04D11A00FC32916A2A
:1041700000290AD001210022AA7659611900FC31D8
:1041800088680028FCD08A6007E00121A976D961FF
:10419000D16C0029FCD00021D164FC339A6A002A3A
:1041A00001D000229A62E0B2FEBD10B50123FFF7F4
:1041B00097FF10BD0300AC3310B5040019706430D4
:1041C00000F0E8FA0123637610BD0000F8B5002284
:1041D0000D0001004276AC31036904000878B1217A
:1041E000C9005850802189005A5001321A629A60E1
:1041F00026006436300000F0DFFA00280ED03000D0
:10420000276900F0CBFA1E4BF8502369FC331A6A79
:10421000002A0CD19A6A002AF9D008E02369002DFF
:104220000AD11A00FC32916A002905D10EE09A6A7F
:10423000002AF3D11A62DBE701225A611A00FC322C
:1042400091680029FCD00021916006E00121D9612C
:10425000D16C0029FCD00021D1641A000020FC326E
:10426000916A81420BD0074990625A5802305A50E5
:10427000824204D0043A534253410230C01AF8BD7E
:104280001C050000C404000010B50121FFF79EFFCB
:1042900010BD000010B51323142202490248FFF795
:1042A000D5FE10BD00400040080F002003210A4841
:1042B00002680A430260094802680A43026008492A
:1042C000084A094B9B1A03DD043BC858D050FBDC5D
:1042D00000F0B4F9FBF74EFF240500405405004000
:1042E0002C7100000000002030010020FEE7FEE7F6
:1042F000FEE7FEE7FEE7FEE7014B18607047C046A9
:104300006C000020F7B50023202877D83C4B8000B4
:10431000C258042A14D006D8022A0DD00ED804237D
:10432000012A14D069E0062A0ED00BD31A2A0DD028
:1043300002231B2A0BD060E0082308E0102306E0CC
:10434000202304E0402302E0802300E001232D4AE3
:104350001268082A04D9092A05D00A21022404E097
:104360000821002401E011000124A02501261C27BA
:104370002548ED004651254D254E2D681B02AD0008
:104380003D400195234D2D6800958559AC46674603
:10439000214D3D401D4385518359C0259C46009BBE
:1043A000AD021D40FF2367461B023B402B43019D8E
:1043B0001D43009B5F0160231F402B003B431C43B8
:1043C00001238451154C036063680F48002BFBD018
:1043D0000024124B01255C60A123DB00C35845601B
:1043E000A025ED0044511BB2914207D002D98A1A90
:1043F000D34003E0521A934000E000231800FEBDB2
:10440000946E0000700000200070004068000020E2
:104410000405000064000020FF00FFFFFC70004066
:10442000F0B520286CD8374B8000C258364B1E6838
:10443000002E2ED1C2243548A4000759344B032541
:104440003B40C0273F023B4303518023893C9B00F4
:10445000FF3C03512F4F03602F4B803CD859FF3C4A
:10446000A043D8510437D859A8432043D85108371E
:10447000D8590C35A843083D2843D851A820C0007E
:104480001E508026C120760280001E501C601E4BEC
:104490001C6000231426214834005C432558040086
:1044A0006F1C0FD1142058432250A0200325C13285
:1044B000FF329200C0051550194A08001268082AF8
:1044C00003D10BE0AA4218D1ECE7082A02D9083A36
:1044D000D14002E00820821A914008001422534380
:1044E000E3189A680C495132FF32920058605050DC
:1044F000DA68C1239B00CA5002E00133032BCBD101
:10450000F0BDC046946E0000C00F002000E100E046
:10451000FF00FFFF04050000009000407400002031
:104520006C0000201E4BF0B5596C18001D4A002984
:1045300014D0A025A12600230124ED05F600D158B2
:104540004F1C06D0D7187F68002F02D027008F405D
:10455000AF5114333C2BF2D100234364131DA0252B
:1045600040329446002001240F4EED05DA680F49D1
:10457000920057180A495218526C002A0CD01A1F80
:104580001268511C05D01968FF2902D02100914002
:10459000A9513A00FC32506414339C45E6D1F0BD79
:1045A000FC900040740000200C05000000900040CA
:1045B00000B5202816D80C4A83009B58032911D82F
:1045C000A0220800C133FF33D2059B0000F014FB8A
:1045D00002080406002104E00C2102E0042100E0AE
:1045E0000321D15000BDC046946E000020280DD894
:1045F000074B8000C058A0220123D2058340002928
:1046000001D1044901E0A121C90053507047C046BF
:10461000946E00000C05000003000020202B0AD837
:10462000A222A021D200C9058858034A9B009B58AA
:10463000D840012318407047946E00002D4B10B5F0
:104640001A78012A19D12C4A1268120715D12B4A5F
:10465000E0241168F0220800104021420BD12849C3
:104660000968114209D12749274A11608021274A48
:104670000902116001E03028F1D01A78012A0DD129
:104680001D490968090709D1F0201C490968014042
:10469000402903D11A490968014223D01B68DBB2C3
:1046A000012B25D1144B1B681B0721D1134B1A6812
:1046B000F0231A40A02A04D1114A12681A4203D0EA
:1046C00016E0D02A14D1F7E7114B1A68012A03D15A
:1046D000C022104B1A600BE00F4A1A601A68012AB8
:1046E000FCD1F5E7C1218020C900C0054250D5E7C3
:1046F00010BDC046E00F00F0E40F00F0E80F00F03E
:10470000EC0F00F0DFFF07C004050040186C00400C
:1047100000EC064014EC064075930000F7B5060067
:104720000D000C008B180193019B671B9C4207D066
:10473000336821781B683000984701340028F3D192
:104740003800FEBD70B505000C00081E07D001F052
:10475000B5F82B6802005B6821002800984770BDFF
:1047600010B5FFF7EFFF10BD10B540220021040087
:1047700000F077FC002320002364636410BD3F2316
:10478000026C10B5541C2340446C9C4201D08154EF
:10479000036410BD0023036443647047436C026CE0
:1047A000934206D03F21C25C01330B4043641000AA
:1047B00001E0012040427047036C406C181A00D59C
:1047C00040307047436C026C934201D0C05C01E002
:1047D000012040427047036C406C5A1C3F23134039
:1047E000181A42424241D0B270470120704710B5BA
:1047F00003681322DB69984710BD70470369054AB7
:104800009950FC331A6A002AFCD0002201201A6257
:104810007047C0461C050000030010B55C331A78D1
:104820001F2313400122110099400D4B0424D96726
:10483000C221036989005C505A60DA60A02200211D
:10484000D20099500122074952425A500649143069
:104850005A500C395A5008315A50FFF79BFF10BD7F
:1048600004E100E00C0500001405000010B5143050
:10487000FFF7A2FF10BD10B51430FFF7A3FF10BD66
:1048800010B51430FFF78AFF10BD0000030070B5AB
:104890005E331C780269604BD45003005D331C7892
:1048A0005E4BD450030061331C785D4B012C0CD15E
:1048B00005005F352E78A225ED00565105006035C4
:1048C0002E78A125ED00565100E00024D450962307
:1048D000DB00994238D996231B01994237D9962398
:1048E0005B01994236D996239B01994234D9E12341
:1048F0009B01994232D99623DB01994231D9E123B8
:10490000DB0199422FD996231B0299422DD9E1232D
:104910001B0299422BD996235B02994229D9E123A4
:104920005B02994227D9E1239B02994225D93D4B4D
:10493000994224D9E123DB02994223D9E1231B03C5
:10494000994221D8384B21E09E23DB021EE09D23B3
:104950001B031BE0354B19E0354B17E0EC239B03A1
:1049600014E0344B12E0344B10E0344B0EE0344B87
:104970000CE0344B0AE0344B08E0344B06E0802373
:10498000DB0403E0324B01E080235B053149002466
:1049900053500423243953501100FC31CC600C6275
:1049A000C1210134890014605C3094605350037855
:1049B0001F202200D9B20840824080342648FF34AC
:1049C0005BB20251002B13DA0F230B40083B234C40
:1049D0009B089B001B1903242140A140FC348C4000
:1049E000DD69A543C0248C4021002943D96111E031
:1049F000194C9B089B001B1903242140A140C02592
:104A0000FC348C40AD005E59A643C0248C4021008C
:104A100031435951026070BD0C05000014050000BF
:104A20006C05000090D0030000D0BE0E00B0130053
:104A30000050270000A04E0000F0750000509D00BF
:104A400000F0EB0000903A0100E0D70100B0AF03A6
:104A500000705F072405000000E100E000ED00E0C9
:104A6000F7B5009308AB1B7800250193FA230400E7
:104A70009B0083600E4B45600833036014300F00C9
:104A80001600FFF771FE23005C3327611E70009B48
:104A9000084A9B00995823005D331970019B200040
:104AA0009B009A5823005E33DD701A70FEBDC0462D
:104AB000186F0000946E0000036910B51A00FC32F4
:104AC000D2680400002A0AD0A322D20099581430D8
:104AD000C9B2FFF754FE00222369FC33DA6010BD2F
:104AE00010B50248FFF7E8FF10BDC046C40F002014
:104AF000162307B5022200930249013B0248FFF743
:104B0000AFFF07BD00200040C40F00207047000029
:104B100010B500F047F8FFF7F9FF012000F024F886
:104B2000FFF790F9FFF7A2F9024B002BFAD000E053
:104B300000BFF7E700000000084A0949094B10B51B
:104B40001B688858FA22190A1B0618439200002392
:104B500000F0D2F94904C00B084310BD0405000061
:104B6000001001402810002070B5041E09D0FFF786
:104B7000E3FF050000F014F8FFF7DEFF401B84425E
:104B8000F8D870BD0022044B9A60044A13680133C0
:104B9000DBB213607047C046FC10014028100020B3
:104BA00070470000C421114A89005058104B03403F
:104BB000C020000203435350802391399B02FF39E8
:104BC000535013608023A3220021DB05D2009950AB
:104BD0000122A1209A60074BC0001950C120023168
:104BE00080001950403019501A60704700E100E011
:104BF000FF00FFFF0010014002B471464908490060
:104C0000095C49008E4402BC7047C046002243083C
:104C10008B4274D303098B425FD3030A8B4244D384
:104C2000030B8B4228D3030C8B420DD3FF220902C6
:104C300012BA030C8B4202D31212090265D0030B85
:104C40008B4219D300E0090AC30B8B4201D3CB037B
:104C5000C01A5241830B8B4201D38B03C01A5241BD
:104C6000430B8B4201D34B03C01A5241030B8B42BF
:104C700001D30B03C01A5241C30A8B4201D3CB02AA
:104C8000C01A5241830A8B4201D38B02C01A52418F
:104C9000430A8B4201D34B02C01A5241030A8B4292
:104CA00001D30B02C01A5241CDD2C3098B4201D3AA
:104CB000CB01C01A524183098B4201D38B01C01A28
:104CC000524143098B4201D34B01C01A524103099F
:104CD0008B4201D30B01C01A5241C3088B4201D34E
:104CE000CB00C01A524183088B4201D38B00C01AFB
:104CF000524143088B4201D34B00C01A5241411A22
:104D000000D20146524110467047FFE701B500202E
:104D100000F0F0F802BDC0460029F7D076E77047F2
:104D200003460B437FD4002243088B4274D303090C
:104D30008B425FD3030A8B4244D3030B8B4228D3AD
:104D4000030C8B420DD3FF22090212BA030C8B42D3
:104D500002D31212090265D0030B8B4219D300E073
:104D6000090AC30B8B4201D3CB03C01A5241830BF8
:104D70008B4201D38B03C01A5241430B8B4201D3A8
:104D80004B03C01A5241030B8B4201D30B03C01AD1
:104D90005241C30A8B4201D3CB02C01A5241830A4B
:104DA0008B4201D38B02C01A5241430A8B4201D37A
:104DB0004B02C01A5241030A8B4201D30B02C01AA4
:104DC0005241CDD2C3098B4201D3CB01C01A52410B
:104DD00083098B4201D38B01C01A524143098B4294
:104DE00001D34B01C01A524103098B4201D30B017D
:104DF000C01A5241C3088B4201D3CB00C01A5241A2
:104E000083088B4201D38B00C01A524143088B4266
:104E100001D34B00C01A5241411A00D201465241FF
:104E2000104670475DE0CA0F00D04942031000D31E
:104E30004042534000229C4603098B422DD3030A73
:104E40008B4212D3FC22890112BA030A8B420CD383
:104E5000890192118B4208D3890192118B4204D3AC
:104E600089013AD0921100E08909C3098B4201D32C
:104E7000CB01C01A524183098B4201D38B01C01A66
:104E8000524143098B4201D34B01C01A52410309DD
:104E90008B4201D30B01C01A5241C3088B4201D38C
:104EA000CB00C01A524183088B4201D38B00C01A39
:104EB0005241D9D243088B4201D34B00C01A524110
:104EC000411A00D20146634652415B10104601D39D
:104ED0004042002B00D54942704763465B1000D327
:104EE000404201B5002000F005F802BD0029F8D0CD
:104EF00016E770477047C046F0B54F464646C0B407
:104F00001604360C9946330005042C0C070C150CBE
:104F100063437E436F4365431C0CAD1964199C4683
:104F2000A64203D980235B02984647446346250C7A
:104F3000EF191D044B464A4343432D0C24046419C6
:104F40009918C91920000CBC90469946F0BDC0467E
:104F50007FB51D000A4B06001B68D868002A02D1E5
:104F6000084C230001E01300074C0293009133002A
:104F70002A000649019400F021F800F011FEC04615
:104F80001001002018690000486F0000556F0000F4
:104F9000084B10B50400002B02D0002100E000BF38
:104FA000054B1868836A002B00D09847200001F059
:104FB000E1FAC04600000000886F00000EB403B59F
:104FC000010003AB044804CB0068019300F016F91C
:104FD00002B008BC03B01847100100200E4B70B59A
:104FE00000251E000D4CE41AA410A54204D0AB000D
:104FF000F35898470135F8E701F0BEFA084B002551
:105000001E00084CE41AA410A54204D0AB00F358CB
:1050100098470135F8E770BD1801002018010020FD
:10502000180100202801002010B5034B010018686A
:1050300000F066F810BDC0461001002010B5034B0B
:105040000100186800F016F810BDC04610010020DD
:10505000002310B59A4203D0CC5CC4540133F9E765
:1050600010BD03008218934202D019700133FAE791
:105070007047000030B500293ED004390B68002B82
:1050800000DAC9181D4A13681400002B02D14B60C6
:10509000116031E08B420DD90A688818834203D130
:1050A00018685B6882180A604B60216024E08A42BD
:1050B00003D813005A68002AF9D11D685C198C4284
:1050C0000BD10968691858181960824214D1106808
:1050D0005268411819605A600EE08C4202D90C23C4
:1050E000036009E008680C18A24203D114685268F2
:1050F000201808604A60596030BDC046301000205A
:10510000032370B5CD1C9D43083506000C2D01D23C
:105110000C2505E0002D03DA0C230020336040E06D
:10512000A942F9D81F4B1C681A002100002913D08E
:105130000B685B1B0DD40B2B02D90B60CC181EE047
:105140008C4202D1636813601AE04B6863600C0004
:1051500016E00C004968E9E7134C2368002B03D1E3
:10516000300000F033FB20602900300000F02EFBFF
:10517000431CD1D00323C41C9C43A0420AD1256008
:10518000200007220B30231D9043C31A09D05A4236
:10519000E25006E0211A300000F018FB431CEED16B
:1051A000BAE770BD301000202C100020936810B5B5
:1051B000013B9360002B05DA9469A34208DBCBB274
:1051C0000A2B05D01368581C10601970C8B201E092
:1051D00000F01AFC10BDF8B506000F001400D51839
:1051E000AC4208D021783A003000FFF7DFFF0134ED
:1051F000431CF5D100E00020F8BD0000F0B59FB0E1
:1052000006000F0002920593002804D08369002B4A
:1052100001D100F0C1FD7F4B9F4201D1776808E0CA
:105220007D4B9F4201D1B76803E07C4B9F4200D188
:10523000F768BB891B070AD53B69002B07D0002301
:1052400006AD6B6120336B761033AB763DE03900F1
:10525000300000F031FC0028F1D001204042D6E0BF
:10526000059A111D12680591002A00DA7FE0099263
:10527000013423782E2B00D18DE021780322684859
:1052800000F070FE002807D0654B2A68C01A402342
:10529000834013432B6001342178631C062261484C
:1052A0000293297600F05EFE002800D19DE05E4B5F
:1052B000002B00D090E00722059B0733934308336F
:1052C00005936B69039A9B186B61029C2378002BF2
:1052D00004D1029BE31A049312D003E0252BF8D0EB
:1052E0000134F3E7049B029A39003000FFF773FFA3
:1052F000431C00D186E06A69049B944663446B6159
:105300002378002B7ED00122002352426A6002A93A
:105310005432521801342B60EB60AB601370AB65F4
:1053200021780522414800F01DFE002808D03F4B9F
:105330002A68C01A0123834013432B600134EFE72E
:105340002B68DA0604D55322202102A81218117006
:105350001A0704D553222B2102A8121811702278A3
:105360002A2A00D17CE7099B00200A2105E052424D
:10537000EA60022213432B607AE72278303A092A46
:1053800004D84B4301349B180120F6E7002800D1D4
:105390006FE709936DE763782A2B0AD1059B0234E6
:1053A0001A1D1B680592002B01DA01235B4207934B
:1053B00063E700230A201A0001346B60217830393A
:1053C000092904D84243013452180123F6E7002B7F
:1053D00000D152E7079250E705AB00933A00144B17
:1053E0002900300000E000BF07E005AB00933A0061
:1053F0000F4B2900300000F08BF80390039B013322
:1054000000D05EE7BB895B0600D526E70B981FB08E
:10541000F0BDC046C0700000E070000000710000E8
:10542000926F0000966F0000000000008C6F00007B
:10543000D7510000F7B5170001938A680B690090F7
:105440000C00934200DA130022003B6043321278D2
:10545000002A01D001333B6023689B0602D53B68DC
:1054600002333B60062523681D401ED023004333D2
:105470001B785A1E9341226892061CD53020E118F1
:105480004331087021005A1C45310978A218433273
:10549000023311700FE022000123193201990098A4
:1054A000089EB047431C0ED00135E3683A689B1A4A
:1054B0009D42F0DBDAE72200019943320098089D13
:1054C000A847431C02D10120404220E00623206867
:1054D000E1683A6803400025042B03D18D1AEB43A1
:1054E000DB171D40A3682269934201DD9B1AED186A
:1054F0000027BD420AD0220001231A3201990098E8
:10550000089EB047431CDED00137F2E70020FEBD05
:10551000F0B58BB006920A004332079305900492CF
:105520000A7E0C00109B6E2A00D1ABE011D8632AD2
:1055300022D009D8002A00D1B5E0582A00D0C5E011
:1055400045310A70814A4FE0642A1DD0692A1BD078
:10555000BCE0732A00D1AAE009D86F2A29D0702AAA
:1055600000D0B3E0202209680A43226037E0752AA0
:105570001FD0782A33D0A9E00E001A684236111DD8
:10558000196013683370A4E021681A68080606D40D
:10559000490604D5111D19600023D55E02E0111DD6
:1055A00019601568002D3BDA2D23049A6D421370A3
:1055B00036E021681A68080606D4490604D515683D
:1055C000111D1960ADB202E0111D196015685F4B25
:1055D000227E039308276F2A1DD00A271BE0220092
:1055E0007821453211705A4A19680392081D2268C1
:1055F00018600D68100602D4500600D5ADB2D3076E
:1056000002D520231A4322601027002D03D1202326
:1056100022689A4322602300002243331A7002E07A
:105620000A274A4B03936368A360002B09DB04221B
:10563000216891432160002D05D1049E002B11D0DB
:105640007BE0002D79D0049E28003900FFF764FB31
:10565000039B013E5B5C280033703900FFF7D6FAEC
:10566000051EF1D1082F09D12368DB0706D5636831
:105670002269934202DC3023013E3370049B9B1B62
:1056800023612BE009681A68080607D4490605D586
:10569000111D19601368A28A1A8004E0111D196097
:1056A000136862691A600023049E236116E01A6879
:1056B000111D1960166800216268300000F052FC6C
:1056C000002801D0801B6060636803E0260042363A
:1056D0003270012323610023049A1370079B09AAE7
:1056E00000932100069B0598FFF7A4FE431C02D1FE
:1056F0000120404227E02369320006990598079D62
:10570000A847431CF4D0236800259B070FD4099BAE
:10571000E068984217DA180015E0220001231932D8
:1057200006990598079EB047431CE1D00135E36810
:10573000099A9B1A9D42F0DBE9E72600039B42365B
:105740001B7833708EE70BB0F0BDC0469D6F000034
:10575000AE6F0000154B10B51C68A36B002B15D164
:105760001820FFF761FC124BA0630380114B01224C
:105770004380114B8380114BC380114B0381052360
:10578000438106338381002302614361A46B0D4A88
:10579000206961690C4BFFF7AFFB012200238018E1
:1057A0005941206161614800400810BD100100208E
:1057B0000E330000CDABFFFF341200006DE6FFFF9B
:1057C000ECDEFFFF2D7F954C2DF45158002370B572
:1057D000064C05000800236000F0B6FE431C03D110
:1057E0002368002B00D02B6070BDC0468C1F0020AA
:1057F0000CB430B5164B9DB00C1E1D6804DA8B231B
:1058000001202B6040421DE0822302A99B008B8176
:105810000023029008619C4200D0631E8B604B61A4
:1058200001235B42CB81209A21AB2800019300F039
:1058300041FC431C01DA8B232B60002C02D0002397
:10584000029A13701DB030BC08BC02B01847C046A5
:10585000100100200EB410B59DB002A9029008619D
:105860000B48822488604861012040421FABC881F8
:10587000084804CBA400006801938C8100F01AFC56
:105880000023029A13701DB010BC08BC03B0184767
:10589000FFFFFF7F1001002002780B78002A03D061
:1058A000013001319A42F7D0D01A7047031C0A78B0
:1058B00001311A700133002AF9D170470023C25C0C
:1058C0000133002AFBD1581E70470000F0B51E00BE
:1058D000454B87B01B680192029308220B0005908C
:1058E00003911C7802995D1C09194878104001D079
:1058F0002B00F6E72D2C04D19D1C5C78012300932E
:1059000004E000902B2C01D15C789D1C002E02D06D
:10591000102E0AD162E0302C5ED120222B789343E6
:10592000582B54D110266C780235009F31007B1E15
:105930009F412E4BFF183800FFF7EEF93800049115
:105940003100FFF763F90023032207009446180093
:10595000029A121951780422114201D0303C07E01A
:105960006246114017D03722012900D02032A41AF4
:10597000A64210DD5A1C0BD0B84207D802D1049BB6
:105980009C4203DC70430123201801E001235B42A9
:105990002C780135DCE75A1C0BD10098059A431E80
:1059A0009841124BC01822231360019B002B0AD18F
:1059B00017E0009A002A00D04042019A002A10D035
:1059C000039A002B00D06A1E019B1A6009E0302464
:1059D000002EAAD10826A8E70A26A6E7302C9CD0DC
:1059E000A3E707B0F0BDC04614010020FFFFFF7F12
:1059F00010B513000A00010002480068FFF766FFB7
:105A000010BDC04610010020F8B505000F001400BD
:105A1000002804D08369002B01D100F0BDF9234B8D
:105A20009C4201D16C6808E0214B9C4201D1AC68DA
:105A300003E0204B9C4200D1EC68A369A360A389DA
:105A40001B070AD52369002B07D023682269FEB201
:105A5000981A636998420FDB08E02100280000F0E3
:105A60002BF80028F1D0012040421DE02100280041
:105A700000F024F90028F6D1A3680130013BA360AF
:105A800023685A1C22601F706369984205D0A3895D
:105A90003000DB0708D50A2E06D12100280000F0CF
:105AA0000DF90028DFD13000F8BDC046C0700000FD
:105AB000E070000000710000354B70B51D680600F5
:105AC0000C00002D05D0AB69002B02D1280000F09E
:105AD00063F9304B9C4201D16C6808E02E4B9C422C
:105AE00001D1AC6803E02D4B9C4200D1EC68A38946
:105AF0009AB2110723D4D10607D4092201203260BB
:105B000037321343A381404240E0530713D5616B02
:105B1000002908D023004433994202D03000FFF717
:105B2000A9FA002363632422A3899343A38100235A
:105B30006360236923600822A3891343A381236937
:105B4000002B0BD1A023A2899B001340802292003E
:105B5000934203D02100300000F0B2F90123A28962
:105B6000134005D00023A36063695B42A36103E097
:105B7000910700D46369A36000202369834205D1A3
:105B8000130603D540231A43A281013870BDC046D5
:105B900010010020C0700000E070000000710000E3
:105BA00010B5062000F0AEFB012000F0E3FC000081
:105BB000F7B58A8905000C0013075AD44B68002BEF
:105BC00002DC0B6C002B19DDE76A002F16D00023D6
:105BD0002E682B6080235B011A4001D0606D14E0B9
:105BE0000123216A2800B847431C0ED12B68002BE3
:105BF0000BD01D2B01D0162B02D12E6000205AE0B5
:105C00004022A3891343A38155E0A3895B0706D5EE
:105C10006368C01A636B002B01D0236CC01A002389
:105C20000200216A2800E76AB847A389421C06D10E
:105C300029681D293AD8204ACA40D20736D5002201
:105C4000626022692260DB0405D5431C02D12B6807
:105C5000002B00D16065616B2E600029CED023003F
:105C60004433994202D02800FFF704FA0020606311
:105C700021E00F69002FC1D00B680F60DB1B01937F
:105C80000023920700D14B69A36003E0019B3F18FA
:105C90001B1A0193019B002BB0DD019B3A00216A86
:105CA0002800A66AB0470028F0DCA3894022012022
:105CB0001343A3814042FEBD010040200B6970B533
:105CC00005000C00002B01D100201CE0002804D0AE
:105CD0008369002B01D100F05FF80B4B9C4201D18E
:105CE0006C6808E0094B9C4201D1AC6803E0084BAA
:105CF0009C4200D1EC680C22A35E002BE4D0210072
:105D00002800FFF755FF70BDC0700000E070000074
:105D10000071000010B5024900F0B0F810BDC04697
:105D2000BD5C0000002310B5040003604360836085
:105D300081814366C2810361436183611900082246
:105D40005C30FFF78EF9054B24626362044BA3625B
:105D5000044BE362044B236310BDC046456300005F
:105D60006D630000A5630000D163000070B5682575
:105D70004B1E5D430E0029007431FFF7C1F9041E6C
:105D800008D000212A00016046600C30A060683213
:105D9000FFF767F9200070BD836913B50400002B7D
:105DA00028D18364C3640365134B144A1B68826261
:105DB0000193984201D101238361200000F020F873
:105DC0006060200000F01CF8A060200000F018F8CF
:105DD0000022E06004216068FFF7A4FF012209218E
:105DE000A068FFF79FFF02221221E068FFF79AFFE9
:105DF0000123A36113BDC046886F0000155D00003C
:105E0000F8B51D4B06001D68AB69002B02D12800B8
:105E1000FFF7C2FF4835AC686B68013B05D40C2224
:105E2000A75E002F10D06834F7E72B68002B01D055
:105E30002D68F0E704213000FFF798FF2860002864
:105E4000F6D10C23336016E0012320005B42E3818E
:105E50000233A38167662760A76067602761676177
:105E6000A7615C3008223900FFF7FBF82000676368
:105E7000A763A764E764F8BD886F0000F7B5040066
:105E80000700002601914834002C16D06368A568ED
:105E90000093009B013B00930DD4AB89012B08D9E3
:105EA0000E22AB5E013304D029003800019B9847D5
:105EB00006436835EDE72468E6E73000FEBD0000E4
:105EC000F0B58B8991B006000C009B0726D40E23F9
:105ED000C95E002904DA8023A5891D4010D10CE099
:105EE00001AA00F0A1FA0028F5DBF023029D1B02B5
:105EF0001D401A4BED186B425D418027FF0001E009
:105F00000025402739003000FFF7FAF800280CD1AF
:105F1000A3899A051FD402221343A3812300473388
:105F2000236023610123636115E080220C4BB3627F
:105F3000A38920601343A38120616761002D0AD0EB
:105F40000E23E15E300000F081FA002803D0012228
:105F5000A3891343A38111B0F0BDC04600E0FFFF49
:105F6000155D0000C9B28218904204D003788B42BC
:105F700002D00130F8E70020704710B5884202D9FE
:105F80008B18984201D3002305E09B1A013A08D3ED
:105F9000995C8154FAE7934203D0CC5CC45401333A
:105FA000F9E710BDF8B506000C001500002904D172
:105FB0001100FFF7A5F8040018E0002A03D1FFF74D
:105FC00059F82C0012E000F067FA85420ED929003A
:105FD0003000FFF795F8071E07D021002A00FFF7D1
:105FE00037F821003000FFF745F83C002000F8BDED
:105FF000F0B58E6885B007000C00039201939E42B5
:1060000043D890238A89DB001A423ED003250969D0
:10601000236801985B1A029363695D43EB0F5D1976
:10602000029B6D1001331B18AB4200D91D005305B4
:1060300010D529003800FFF763F8061E14D0029A25
:106040002169FFF705F8A289194B134080221343F9
:10605000A38112E02A003800FFF7A4FF061E0CD12E
:1060600021693800FFF706F80C23402201203B602D
:10607000A38940421343A38117E0029B2661F618CF
:1060800026606561019EED1AA560019BB34200D2B6
:106090001E00320003992068FFF76FFF0020A368FD
:1060A0009B1BA36023689E19266005B0F0BDC04607
:1060B0007FFBFFFFF0B59FB0029005938B890F0027
:1060C00016001B0610D50B69002B0DD14021FFF7E0
:1060D00017F838603861002804D10C23029A01387F
:1060E0001360D8E040237B61002306AD6B61203351
:1060F0006B761033AB7634002378002B03D1A31BCF
:10610000049312D003E0252BF9D00134F4E7A31B4C
:10611000320039000298FFF76BFF431C00D1B4E056
:106120006A69049B944663446B612378002B00D119
:10613000ABE00122002352426A6002A95432521895
:1061400001342B60EB60AB601370AB65534E21786C
:1061500005223000FFF706FF002807D00123801B2F
:1061600083402A68013413432B60EFE72B68DA067B
:1061700004D55322202102A8121811701A0704D541
:1061800053222B2102A81218117022782A2A03D038
:10619000099B00200A210EE0059A111D1268059145
:1061A000002A01DB099204E05242EA600222134312
:1061B0002B6001340BE02278303A092A04D84B4393
:1061C00001349B180120F6E7002800D009932378BA
:1061D0002E2B1ED163782A2B0AD1059B02341A1D5F
:1061E0001B680592002B01DA01235B42079310E044
:1061F00000230A201A0001346B6021783039092904
:1062000004D84243013452180123F6E7002B00D092
:106210000792234E217803223000FFF7A3FE0028C7
:1062200006D04023801B83402A68013413432B602F
:10623000217806221B48661C2976FFF793FE00286A
:1062400012D0194B002B06D10722059B073393432D
:106250000833059314E005AB00933A00134B290073
:10626000029800E000BF07E005AB00933A000F4B37
:1062700029000298FFF74CF90390039B013304D0E7
:106280006B69039A9B186B6135E7BB890B985B06BA
:1062900001D5012040421FB0F0BDC0468C6F000008
:1062A000926F0000966F000000000000F15F000098
:1062B00070B504000D1E1F2D04D9162303600120A4
:1062C00040421EE0426C002A04D08B00D2181368B2
:1062D000002B08D1200000F031F82A000100200036
:1062E00000F01AF80DE00020012B0AD0591C03D150
:1062F00017332360013004E000242800146098471D
:10630000200070BD10B5034B01001868FFF7D0FFE7
:1063100010BDC04610010020002370B5064C0500DA
:1063200008001100236000F0F7F8431C03D1236834
:10633000002B00D02B6070BD8C1F002010B500F02A
:10634000DBF810BD70B50C000E25495F00F0B0F809
:10635000002803DB636D1B18636503E0A289024B11
:106360001340A38170BDC046FFEFFFFFF8B51F00CB
:106370008B8905000C001600DB0505D50E23C95ED0
:106380000022022300F074F8A289054B2800134074
:10639000A38132000E23E15E3B0000F01FF8F8BD40
:1063A000FFEFFFFF70B50C000E25495F00F060F8AD
:1063B000A389421C03D1054A1340A38104E0802233
:1063C00052011343A381606570BDC046FFEFFFFF1C
:1063D00010B50E23C95E00F015F810BD70B50500AC
:1063E000080011000022064C22601A0000F0BAF8E2
:1063F000431C03D12368002B00D02B6070BDC04626
:106400008C1F0020002370B5064C05000800236097
:1064100000F062F8431C03D12368002B00D02B60EE
:1064200070BDC0468C1F0020002370B5064C0500CF
:1064300008001100236000F057F8431C03D12368C3
:10644000002B00D02B6070BD8C1F0020002370B586
:10645000064C05000800236000F056F8431C03D1E9
:106460002368002B00D02B6070BDC0468C1F00201D
:1064700070B50500080011000022064C22601A00C9
:1064800000F052F8431C03D12368002B00D02B608E
:1064900070BDC0468C1F00200B1F1A68101F002AF9
:1064A00004DA891804390B68D018043870470000E2
:1064B00070B50500080011000022064C22601A0089
:1064C00000F03AF8431C03D12368002B00D02B6066
:1064D00070BDC0468C1F002058220120014B404255
:1064E0001A6070478C1F002058220120014B404247
:1064F0001A6070478C1F002058220120014B404237
:106500001A6070478C1F00205822024B00201A602E
:106510007047C0468C1F002058220120014B40428A
:106520001A6070478C1F002058220120014B404206
:106530001A6070478C1F002058220120014B4042F6
:106540001A6070478C1F0020044A1368002B03D088
:106550001818106018007047014BF9E7341000203C
:10656000901F002058220120014B40421A607047C2
:106570008C1F0020FEE7C046F8B5C046F8BC08BC3A
:106580009E467047F8B5C046F8BC08BC9E467047AA
:1065900066616C73650074727565006C6973742054
:1065A0006F66202564206974656D73006F626A658B
:1065B0006374206F6620636C6173733A20256400F6
:1065C000537461636B20756E646572666C6F7700DF
:1065D000B80600004C060000C2060000F8060000E5
:1065E000340700006E070000AA070000D60700006D
:1065F000140800005A080000B6080000FC0800005B
:106600006A090000B8090000E40900001E0A000041
:10661000680A0000900A0000C20A0000F80A0000A0
:10662000320B0000B80B00007E0C0000040D0000CF
:10663000600D0000A20D0000C40D0000CC0D000094
:10664000AE0E0000B8060000B8060000B806000054
:10665000B8060000B8060000B8060000FA0E0000F8
:10666000440F0000920F000018100000B610000048
:10667000041100004E11000094110000E011000010
:106680002C12000078120000C41200001013000049
:106690004E130000BA130000EA130000401400007B
:1066A0008C140000D8140000121500005E150000C4
:1066B000B8060000B8060000B8060000B8060000E2
:1066C000AA150000DA1500000A16000036160000B0
:1066D0006616000092160000B8060000B80600001A
:1066E000B8060000B8060000C21600000A17000035
:1066F0005617000086170000B2170000F4170000BC
:10670000B8060000B8060000B8060000B806000091
:10671000341800006418000094180000C418000029
:10672000F0180000201900004C1900007619000034
:10673000A0190000D0190000001A00002C1A000057
:10674000581A0000881A0000B41A0000B8060000A9
:10675000B8060000B8060000B8060000B806000041
:10676000E41A0000101B00003C1B0000681B000026
:10677000A41B0000D41B0000041C0000341C0000FB
:10678000641C0000901C0000BE1C0000EE1C0000F9
:106790001C1D00005C1D0000941D0000B8060000D8
:1067A000B8060000B8060000B8060000B8060000F1
:1067B000B8060000B8060000B8060000B8060000E1
:1067C000B8060000B8060000C21D0000F01D000061
:1067D0000D0A564D2050616E69633A2025730D0AEB
:1067E00000496E73756666696369656E74206D65D0
:1067F0006D6F727920666F72204D6963726F426CA3
:106800006F636B73206F626A656374206865617083
:1068100000496E73756666696369656E74206D659F
:106820006D6F727920666F72204D6963726F426C72
:106830006F636B7320737461636B00626164206FBC
:10684000626A65637420617420256C640A0025788F
:106850003A20256420776F7264732C20636C617317
:106860007349442025640A004865616465723A20D2
:1068700025780A0009307825782C0A00256420251F
:10688000642025642025640A0042616420726563E7
:106890006F726420666F756E6420647572696E67CE
:1068A00020696E697469616C697A6174696F6E21BF
:1068B0000A004E6F7420656E6F75676820726F6F87
:1068C0006D206576656E20616674657220636F6DFC
:1068D00070616374696F6E0A00526573746F7269D8
:1068E0006E6720256420736372697074732E2E2E78
:1068F0000053746172746564002D2D2D2D2D0A00D6
:1069000050657273697374656E74204D656D6F7236
:106910007920546573740A0A000A496E69746961C2
:106920006C697A696E67204D656D6F72790A004DEA
:10693000656D6F727920696E74697469616C697ACA
:1069400065643B2077726974696E67207265636F56
:106950007264732E2E2E0A005265636F726420617A
:1069600074206F66667365742025643A2025642060
:1069700025642025642025642028256420776F72F3
:106980006473290A0046696E616C3A2063757272FD
:10699000656E74202564207573656420256420630A
:1069A000302025642063312025640A004E6F206664
:1069B000726565207461736B20656E7472696573AE
:1069C0000057656C636F6D6520746F204D6963724D
:1069D0006F426C6F636B7321004D656D6F72792030
:1069E000636C65617265642E00416C6C2074617328
:1069F0006B732073746F707065640076303433008D
:106A0000202573202573000007000000030000000C
:106A10006D6963726F3A62697400696F00686173CF
:106A2000546F6E6500706C6179546F6E65006861BB
:106A300073536572766F00736574536572766F0079
:106A40000000000001000000020000000300000040
:106A5000040000000A0000006E6574007374617227
:106A6000745769466900697357694669436F6E6E6A
:106A70006563746564006D7949504164647265733F
:106A800073007468696E67446573637269707469D2
:106A90006F6E00636C6561725468696E67446573FC
:106AA0006372697074696F6E00617070656E6454B2
:106AB0006F5468696E674465736372697074696F57
:106AC0006E001A1B1C03040607090A1718191A1B63
:106AD0001C030406646973706C6179006C696768F3
:106AE000744C6576656C0000000000000100000039
:106AF0000200000003000000040000000500000088
:106B00000600000007000000080000000900000067
:106B10000A0000000B0000000C0000000D00000047
:106B20000E0000000F000000100000001200000026
:106B30001400000016000000180000001A000000F9
:106B40001C0000001E0000002000000023000000C8
:106B500026000000290000002C0000002F0000008B
:106B600032000000360000003A0000003E00000045
:106B700042000000460000004B00000050000000F2
:106B8000550000005A00000061000000680000008D
:106B90006F000000760000007D000000840000000F
:106BA0008B0000009200000099000000A00000008F
:106BB000A7000000AE000000B5000000BC0000000F
:106BC000C3000000CA000000D1000000D80000008F
:106BD000DF000000E6000000ED000000F40000000F
:106BE000FB000000FF000000000000000008080893
:106BF00000080A4A4000000A5FEA5FEA0ED92ED375
:106C00006E19324489330C924C924D0808000000F2
:106C100004880808040804848488000A448A400020
:106C2000048EC480000000048800000EC000000034
:106C300000080001224488100C9252524C048C84AB
:106C4000848E1C824C901E1EC244924C06CA525F17
:106C5000E21FF01EC13E02448ED12E1FE244881076
:106C60000ED12ED12E0ED12EC488000800080000AF
:106C7000048004880244880482000EC00EC0080408
:106C80008244880ED126C0040ED135B36C0C925EBE
:106C9000D2521C925C925C0ED010100E1C9252527A
:106CA0005C1ED01C901E1ED01C90100ED013712E96
:106CB00012525ED2521C8808081C1FE242524C122B
:106CC00054981492101010101E113B75B1311139E7
:106CD00035B3710C9252524C1C925C90100C925233
:106CE0004C861C925C92510ED00C825C1FE4848412
:106CF00084125252524C1131312A44113135BB7138
:106D000012524C9252112A4484841EC488101E0EC2
:106D1000C808080E10080482410EC242424E048A7E
:106D2000400000000000001F0804800000000ED298
:106D3000524F10101C925C000ED0100E02424ED228
:106D40004E0C925C900E06C81C88080ED24EC24CA7
:106D500010101C92520800080808024002424C1011
:106D6000149814920808080806001B75B131001C1D
:106D7000925252000C92524C001C925C90000ED227
:106D80004EC2000ED010100006C8049808080EC8A5
:106D900007001252524F0011312A4400113135BB05
:106DA00000124C8C9200112A4498001EC4881E06C2
:106DB000C48C8486080808080818080C8818000085
:106DC0000C8360535049436C6173733A3A53504992
:106DD000436C617373284E52465F5350495F547938
:106DE00070652A2C2075696E74385F742C20756963
:106DF0006E74385F742C2075696E74385F74290066
:106E0000705F73706920213D204E554C4C002F550A
:106E1000736572732F6A6F686E6D616C6F6E6579E2
:106E20002F4C6962726172792F41726475696E6F5D
:106E300031352F7061636B616765732F73616E64A9
:106E40006565706D69737472792F686172647761BA
:106E500072652F6E5246352F302E362E302F6C69CC
:106E6000627261726965732F5350492F5350492ED6
:106E70006370700000000000000000001B40000074
:106E8000E13F0000074000001140000041400000C9
:106E900005400000030000000200000001000000A7
:106EA0000400000005000000110000000C000000BC
:106EB0000B000000120000000A00000006000000A5
:106EC0001A00000014000000170000001600000067
:106ED0001500000010000000FFFFFFFFFFFFFFFF95
:106EE000000000001E000000190000001800000053
:106EF0000700000008000000090000000D0000006D
:106F00000E0000000F0000001C0000001B0000002D
:106F10001D00000013000000000000000000000041
:106F2000FD4700001D4700006D480000814800003B
:106F300077480000FB470000EF4700008D48000045
:106F400019480000EB4700002C2066756E637469D9
:106F50006F6E3A2000617373657274696F6E2022E0
:106F6000257322206661696C65643A2066696C65E8
:106F700020222573222C206C696E652025642573E0
:106F800025730A0043000000B0000020232D302BA1
:106F90002000686C4C00656667454647003031321A
:106FA0003334353637383941424344454600303171
:106FB00032333435363738396162636465660000D0
:106FC0002020202020202020202828282828202099
:106FD00020202020202020202020202020202020B1
:106FE0008810101010101010101010101010101029
:106FF0000404040404040404040410101010101009
:1070000010414141414141010101010101010101E1
:107010000101010101010101010101101010101015
:1070200010424242424242020202020202020202B2
:1070300002020202020202020202021010101020DA
:107040000000000000000000000000000000000040
:107050000000000000000000000000000000000030
:107060000000000000000000000000000000000020
:107070000000000000000000000000000000000010
:107080000000000000000000000000000000000000
:1070900000000000000000000000000000000000F0
:1070A00000000000000000000000000000000000E0
:1070B00000000000000000000000000000000000D0
:1070C00000000000000000000000000000000000C0
:1070D00000000000000000000000000000000000B0
:1070E00000000000000000000000000000000000A0
:1070F0000000000000000000000000000000000090
:10710000000000000000000000000000000000007F
:10711000000000000000000000000000000000006F
:04712000000000006B
:087124005090FF7F0100000004
:10712C00FFFFFFFF1D6A0000F1300000256A000020
:10713C00ED3000002E6A0000F5300000376A0000C8
:10714C00F93000005C6A0000C5330000666A00007C
:10715C00CF330000766A0000D9330000826A000049
:10716C00A5330000936A0000B9330000A96A00003F
:10717C00AF330000DC6A000015340000180000007A
:10718C00FF000000030000000200000008000000E7
:10719C000A000000FFFFFFFF0000000001000000DC
:1071AC000000020001000000FFFFFFFF00000000D4
:1071BC00020000000000040002000000FFFFFFFFBF
:1071CC0000000000030000000000080003000000A5
:1071DC0000000000C0700000E070000000710000B2
:1071EC000000000000000000000000000000000093
:1071FC00846F000000000000000000000000000090
:10720C000000000000000000000000000000000072
:10721C000000000000000000000000000000000062
:10722C000000000000000000000000000000000052
:10723C00B0000020BF6F000039010000B13F00001A
:10724C0095420000F14A00000D0100000000000012
:04000003000042AD0A
:00000001FF
